:020000040100F9
:1000000038480020E5000001ED000001EF0000018C
:1000100000000000000000000000000000000000E0
:10002000000000000000000000000000F1000001DE
:100030000000000000000000F3000001F5000001D6
:10004000F7000001F7000001F7000001F7000001D0
:10005000F7000001F7000001F7000001F7000001C0
:10006000F7000001F7000001F7000001F7000001B0
:10007000F7000001F7000001F7000001F7000001A0
:10008000F7000001F7000001F7000001F700000190
:10009000F7000001F7000001F7000001F700000180
:1000A000F7000001F7000001F7000001F700000170
:1000B000F7000001F7000001F7000001F700000160
:1000C0000348854600F056F80048004751050001F6
:1000D0003848002040BA7047C0BA70470138FDD197
:1000E000704700000448804704480047FEE7FEE7E9
:1000F000FEE7FEE7FEE7FEE795030001C100000111
:1001000030B50B46014600202022012409E00D46AF
:10011000D5409D4205D31D469540491B2546954037
:1001200040191546521E002DF1DC30BD03460B432D
:100130009B0703D009E008C9121F08C0042AFAD29D
:1001400003E00B780370401C491C521EF9D2704723
:10015000D2B201E00270401C491EFBD2704700225F
:10016000F6E710B513460A4604461946FFF7F0FFB6
:10017000204610BD064C0125064E05E0E36807CC7D
:100180002B430C3C98471034B442F7D3FFF79CFF45
:10019000C0070001D0070001F7B5D4B004460E46F1
:1001A00000205390052052900025002700BFEFF358
:1001B00010800090FF21453101A8FFF7D0FF00F02B
:1001C000F1F905462448854218D1012000038442F4
:1001D00002D1002053902AE001204003844202D142
:1001E0004011539023E003200003844203D10120F7
:1001F000400253901BE0529857B0F0BD174885421B
:1002000013D101200003844201D153900FE001205B
:100210004003844201D1539009E00320000384424B
:1002200001D1539003E05298E6E75298E4E705AF16
:100230000137FF2241320A4901A8FFF777FF012069
:1002400000F04FF93146569A5398B84752900098AB
:1002500000F047F95298CFE7C440130085601300BF
:10026000E8050001F1B58AB0002009907D20C000AA
:1002700008900125AD020027002007907F200690FE
:1002800040240026002005900390200102900020C9
:1002900001903E490A98884206D83D4800686102AC
:1002A00088433B49086006E0394800680121C903DA
:1002B0000843374908607D21C9000A98FFF720FFED
:1002C0007D21C9000090FFF71BFF450100BF3048AA
:1002D00000687F21090288430190200201990843A8
:1002E0002B4908600520FFF7F9FE10E00120FFF719
:1002F000F5FE2748406B02210840002800D007E0A7
:100300000598411C05910899884200D900E0EDE765
:1003100000BF1F48C06B86B2AE4201D9771B00E018
:10032000AF1B0298874203D2E0B20390B8B20290AA
:10033000AE4201D3069400E007940699079840184E
:10034000C005000E04900498A04200D103E0049C74
:1003500009988742BBD800BF0D4800687F21090279
:1003600088430190039800020199084308490860F6
:100370000846406840084000486000BF04484068A4
:10038000042108400028F9D10BB0F0BD0090D00343
:100390000010024010B53E48C0690121090708431A
:1003A0003B49C861812000063A4908633A484861E0
:1003B0003A4808623A48006803218903884338496B
:1003C00008603421374800F073F836480069401C53
:1003D000002803D033480069002817D12C48406812
:1003E0000121090408432A4948600846406807215A
:1003F00009028843264948600846406809150843B1
:10040000234948602848FFF72DFF3FE021488069D5
:100410004409640123480078C006C00E04431D4807
:1004200084611B4800680121C9038843184908609A
:10043000084600687F21090288430446194800697C
:10044000000220431249086008464068012109045F
:1004500008430F494860084640680721090288435D
:100460000B49486008464068091508430849486038
:100470000846006A0D490840054908620846006AB6
:100480000849C968090208430149086210BD000013
:1004900000100240007000400F0800001800020029
:1004A00000100140004000200090D003FF00F8FF42
:1004B00070B504460D462A46214601200003FFF789
:1004C0006BFE70BD02E008C8121F08C1002AFAD1F5
:1004D00070477047002001E001C1121F002AFBD1C4
:1004E000704780F31088704730B502460B460021F4
:1004F000C94312E01078521C414000240BE0480828
:10050000CD07ED0F002D01D0074D00E0002568401C
:100510000146601CC4B2082CF1DB18465B1E0028A3
:10052000E8D1C84330BD00002083B8ED0446012067
:10053000C007204305490863206880F3088800BF8E
:1005400062B66068804700BFFEE7000000700040B0
:10055000114C124D1249206888421AD12821204698
:10056000FFF7C2FFA16A884213D16168022902D154
:100570002146183101E0214608310846074A016842
:10058000914205D32122D2040168914200D205682C
:1005900000BF2846FFF7CAFF0040000100800001AD
:1005A00011C011CA70B5D2B00024002500BFEFF30E
:1005B00010800646FF21453101A8FFF7D0FD01ACB0
:1005C00001349822074901A8FFF7B0FD0120FFF789
:1005D00088FFA04705463046FFF783FF284652B004
:1005E00070BD00002807000140BA7047C0BA7047CC
:1005F0000138FDD170470000F7B50325AD06286A24
:1006000082B016460C46400840002862286A022143
:1006100008432862286A8007FCD4662068600127A6
:100620002F61A86AC005FCD5992068602F61A86A6F
:10063000C005FCD5FF209130FFF7DAFFFF2301331F
:10064000AB626846EF60352169602F61A96AC90510
:10065000FCD5AB62A969EF60C9B205226A602F615F
:10066000AA6AD205FCD5AB62AA690902D2B21143CB
:100670000180C80702D0032005B0F0BDAB626869F5
:10068000FF210831884368616869C91E08436861B1
:1006900002980002483068600820A860EE602F6170
:1006A000A86AC005FCD5FF200130A8620023F61C13
:1006B000B0080ED0B2081148006899006054060ACC
:1006C00009194E70060C000E8E705B1CC8709A42A1
:1006D000F1D8FF200130A8626869FF210831884302
:1006E0006861686938436861286A80088000286208
:1006F000286A38432862002005B0F0BD8000000C55
:10070000032080064169FF2208329143416142691A
:1007100001210A434261026A920892000262026A5F
:100720000A43026270470000002003218906096A1B
:10073000490849000322920611621146096A022201
:10074000114303229206116200BF03218906096A40
:10075000022211400229F8D0D101032292069162AF
:100760000321D1609F2151600121116100BF03214C
:100770008906896AFF22013211409142F7D1032292
:1007800092069162114688694969FF2208329143B5
:100790000322920651611146496901221143032245
:1007A000920651611146096A890889001162114651
:1007B000096A012211430322920611627047000068
:1007C000D00700010040002038080000D4040001D8
:1040000011C011CA01000000008000010C9B0000DB
:10401000D89057F1000000000000000000000000F0
:0C402000000000000000000060D396EDDE
:1080000000B100206981000171810001999800018F
:108010000000000000000000000000000000000060
:108020000000000000000000000000005D9C000156
:10803000000000000000000027810001619C000199
:108040007B8100017B8100017B8100017B8100013C
:108050007B8100017B8100017B8100017B8100012C
:108060007B8100017B8100017B8100017B8100011C
:108070007B8100017B8100017B8100017B8100010C
:108080007B8100017B8100017B8100017B810001FC
:108090007B8100017B8100017B8100017B810001EC
:1080A0007B8100017B8100017B8100017B810001DC
:1080B000699E00017B8100017B8100017B810001C1
:1080C0000348854600F0D0FC0048004769D4000111
:1080D00000B1002040BA7047C0BA70470138FDD1E6
:1080E0007047000040BA7047C0BA7047704670478A
:1080F000084B19680868203080F30988022080F353
:108100001488BFF36F8F3FBCAE4608BC04BC62B698
:108110001847000084470020EFF3108072B67047C4
:1081200080F310887047EFF309800E4B1A682038EF
:108130001060F0C044464D4656465F46F0C008B554
:1081400072B607F091FD62B60CBC11680868103079
:10815000F0C8A046A946B246BB4680F3098820383D
:10816000F0C8184784470020044880470448004767
:10817000FEE7FEE7FEE7FEE7FEE7FEE7B99C00014B
:10818000C180000130B50B460146002020220124A9
:1081900009E00D46D5409D4205D31D469540491B3B
:1081A0002546954040191546521E002DF1DC30BD84
:1081B00070B500242546002801DA01244042002938
:1081C00001DA01254942FFF7DDFFAC4200D0404211
:1081D000002C00D0494270BDF0B51FB40646002007
:1081E00082B005464024019100901BE0019922468F
:1081F0000F46304600F060FB049A059B801A9941B7
:1082000010D310461946224600F046FB361A8F411D
:108210000197224601200021009F00F03DFB381805
:108220004D4100902046641E0028DFDC019B009831
:108230002946324607B0F0BD0549064A0868504352
:10824000054A801808604008704701490860704777
:10825000DC4700206D4EC6413930000003460B4319
:108260009B0703D009E008C9121F08C0042AFAD2EC
:1082700003E00B780370401C491C521EF9D2704772
:10828000D2B201E00270401C491EFBD270470022AE
:10829000F6E710B513460A4604461946FFF7F0FF05
:1082A000204610BD421C0178401C0029FBD1801AD9
:1082B000704710B5002200E0521C835C8C5CA34226
:1082C00001D1002BF8D1D8B2E1B2401A10BDC9B229
:1082D00003E003788B4203D0401C521EF9D20020E9
:1082E000704730B504460020034600E05B1C934213
:1082F00003D2E05CCD5C401BF8D030BD03460A7869
:108300000270401C491C002AF9D11846704730B54C
:1083100005460020034600E05B1C934205D2EC5C5E
:10832000C85C201A01D1002CF6D130BDF8B5024648
:108330004A40D40F42004B0052085B089A4202D2D6
:108340000246084611464A0023D0C30D4A00DDB25A
:10835000120EAD1A202D35DA49020126490AF6051A
:108360008A19002C00D0524220214F1B1146B940DF
:108370002A411018C20D9A4221D0002C17D0012D8D
:1083800008DCDA05801AD20F8019D207DBB200F0C0
:10839000BFFAF8BDDA05801A012340001B06C01899
:1083A00080185A428018CA0F1043490007E0490854
:1083B000C2071143DA05801A80194008801800F0BE
:1083C0009FFAF8BD61000122511A001BF7E7012254
:1083D000D2075140AAE70122D2075040A6E7024641
:1083E00070B54A40D30FDB0740002DD04A002AD099
:1083F000010E140E000212020919400A520A8418D2
:10840000E50104465443000A120A2E045043A419FD
:108410004219200CC543AA18120C0125AD03521CA9
:10842000521912047F39240400D0521C104301D485
:108430004000491EC2B20C06C0092018401C40086A
:10844000802A02D003E0002070BD400840000029CF
:1084500000DA0020184370BDF0B5074608465840C2
:1084600087B0C00F049048000E46590040084908E4
:10847000BC1A884105D2384631461E4617460B467F
:1084800002465800400810434CD0300D0390400580
:108490005900400D490D0590401A0290402872DAAB
:1084A00018030121000B090508430190049800926C
:1084B000002805D001995242002088410092019085
:1084C000029840210A1A0199009800F0E5F9054642
:1084D0000C466B4607CB00F000FAC0197141039AB5
:1084E0000E0D0023D71756401A467A40164344D043
:1084F000049A002A2DD0029A012A039A15DC12054B
:10850000C01A914101263605001C7141D20F059E0B
:10851000D2070093019202962A46234600F03EFAC3
:1085200007B0F0BD38463146FAE71605224A0F4635
:10853000B218C01AB74101210905001C4F410018AB
:108540007F41114618187941E20F10436D196441BB
:1085500013E0E2076D0815436408C2071443039A49
:1085600001261205C01A91413605001C7141CE0743
:10857000400830434908C01851412A46234600F0BC
:1085800000FACDE7FFE7049801224000C117121A54
:1085900000238B4104983146C417381AA141EEE7F5
:1085A00030B40124E407634030BC55E730B4012403
:1085B000E407614030BC4FE70000E0FFF0B51FB4B6
:1085C00088B00B990998002448400999C00F4900C8
:1085D00049080991C0070B990090490049080B917F
:1085E00009990898A64608431CD00B990A98084395
:1085F00018D0099801244000420D4800410D099807
:1086000024050003000B204309900B980003000B86
:1086100020430B9050181C4940180022019014462A
:10862000104605E0002001460DB0F0BD032801DA38
:10863000034600E003239C46C11A0AAE0AE05F002D
:1086400008ADED5B4F00F75B7D430027AA187C4126
:10865000491C5B1E6145F2DD410004AB5A52210406
:10866000120C0A43240C401C0828DFDB01980290FE
:108670000099704601910090059B049A079906980D
:1086800000F08CF9D0E700000DFCFFFFF0B50C46C0
:108690005C4085B0E40FE40703944C0000266408B6
:1086A00059009446490802460296224321D0624668
:1086B0000A431ED06200570D4A000E032303550DD6
:1086C000012402462C492405781B1B0B360B40184D
:1086D00023432643614600901C46501AB44103D3FD
:1086E0000098401C009002E0921800985B4100281E
:1086F00003DA0020014605B0F0BD00200121090584
:108700000746864611E064461D46141BB54106D354
:108710006546521BB341744607430C43A646CD073A
:1087200040084908284392185B4105460D43EAD1A9
:108730001046184313D06046194650407140084314
:1087400006D06046101AB34106D20122002306E08B
:1087500000220123DB0702E00122D24353100098DC
:1087600074460105381C6141029C039D0019694152
:1087700000F007F9BFE70000FD03000010B500227C
:108780009623114600F0C4F810BD00000EB505494F
:108790000291002100910A460B46019100F0FEF87B
:1087A00003B000BD330400000EB5054A029200225A
:1087B00000921346019200F0F1F803B000BD0000F2
:1087C00033040000C20F410040020123400ADB05D0
:1087D000D207090EC0187F2901DA002070479629B8
:1087E00003DC9623591AC84001E096398840002AD4
:1087F000F4D04042704700004A0009030123090BEE
:108800001B0519430A4B10B5520D9A4202DA00209B
:10881000014610BD064B34339A4203DC9A1A00F02D
:108820004BF810BD034BD21800F036F810BD000015
:10883000FF030000CDFBFFFFC20FD207400040083E
:108840000BD0C10D0723DB01C91840020905400AFE
:108850001143C2084007114370470020014670478A
:10886000CB0FDB07490010B5490802460A4307D081
:108870000A0D07240903E401090B121B002A01DC7D
:10888000002010BDC900440F0C43C100E018D20500
:10889000801800F035F810BD10B5202A04DB014621
:1088A000203A9140002010BD914020239C1A03469D
:1088B000E3401943904010BD10B5202A04DB084660
:1088C000203AD040002110BD0B46D340D040202498
:1088D000A21A91400843194610BD10B5202A06DBA4
:1088E000CB170846203A1041C1170B4306E00B4650
:1088F0001341D0402024A21A91400843194610BDCC
:10890000002904DA401C490001D1400840007047AA
:1089100070B40024050C05D11024000402D10029F4
:1089200021D01124050E01D100020834050F01D118
:108930000001241D850F01D18000A41C002801DB4B
:108940004000641C002908D020252E1B0D46F54050
:10895000A14000D001212943084301061B1B000A46
:10896000DB1D02D5002070BC7047DB05181880188D
:108970000029F8DA401C4900F5D170BC40084000DD
:10898000704710B5002B08DA0024401C6141921892
:108990005B411A4301D14008400010BDF0B51FB43F
:1089A00082B005460C0003D0084601F03FFB02E010
:1089B00001F03CFB20300246009021462846FFF79C
:1089C0006BFF049B059A04460F4618431143084366
:1089D00014D0184610431BD0009840210A1A18469C
:1089E0000599FFF769FF05460E46009A0599049818
:1089F000FFF752FF084305D0012004E02046394626
:108A000007B0F0BD0020C11705430E432C43374388
:108A100000990E986305401A7905E40A00220C4378
:108A2000FD0A0A3002D500200146E9E701051019C8
:108A300069410C9C0D9D00196941FFF7A2FFDFE71A
:108A400010B5002904DB0124E40740428C41214693
:108A5000002B04DB1C460123DB075242A341994251
:108A600000D1904210BD0000064C0125064E05E0E5
:108A7000E36807CC2B430C3C98471034B442F7D33F
:108A8000FFF722FBEC1401010C15010170B58D18E4
:108A90000478401CA207920F01D10278401C2311D8
:108AA00006D10378401C03E006780E70401C491C78
:108AB000521EF9D1002B15D002780C268A1A3440A8
:108AC000401C0C2C03D0A401121B9B1C08E0047852
:108AD0002402121B401CF8E714780C70491C521C2D
:108AE0005B1EF9D5A942D3D3002070BD03B4014861
:108AF000019001BD232A000003B40148019001BD8B
:108B00006D56000003B40148019001BD656000008E
:108B100003B40148019001BDAF7F000003B40148D8
:108B2000019001BDB551000003B40148019001BDA1
:108B3000D37E000003B40148019001BD697E0000AE
:108B400003B40148019001BDC37F000003B4014894
:108B5000019001BDE954000003B40148019001BD3A
:108B60009957000003B40148019001BDED57000082
:108B700003B40148019001BD1D7C000003B401480D
:108B8000019001BDAB52000003B40148019001BD4A
:108B9000F58F000003B40148019001BDE1FE000023
:108BA00003B40148019001BD250E010003B4014842
:108BB000019001BDB143000003B40148019001BD23
:108BC00085290000C943416070470268702392B252
:108BD0009A430A430260704770B5044601F02CF9CD
:108BE000002818D08069002815D0FFF7C7FD05467A
:108BF0002046FFF7C3FD2946FFF7EDFBFFF71CFEFC
:108C0000064A074BFFF742FD0022064BFFF724FC04
:108C1000FFF726FE70BD044DEAE700001F85EB510B
:108C2000B81E01400000394000803B4470B50D463D
:108C30000646002401F000F9002816D0C169002979
:108C400013D0026A002A10D08BB290B289B292B2CD
:108C5000102D0CD0202D0AD0302D17D0402D15D03E
:108C6000502D13D0602D11D022E0002070BD891A44
:108C7000B01AAF2292005043FFF79AFA0446963496
:108C80000FD47D20C000844211DC11E0191AAF22FC
:108C9000301A12015043FFF78BFA4B21C9004418D8
:108CA00001D5002404E0E1200001844200DD0446F7
:108CB000204670BD70B5104CA0421BD18514012117
:108CC000284600F06BFF0021284600F067FF0121D5
:108CD000284600F057FF094860610020206060606E
:108CE0001F21A16006492161A06160622062A0622B
:108CF0000448E06170BD000000080240080A02005C
:108D00000000FC0F2E6D00000029016802D0012236
:108D1000114301E04908490001607047042200291D
:108D2000816902D011438161704791438161084894
:108D30000649C162074901630749416307498163E5
:108D40000749C16308490748086070472200780056
:108D500000080240E700E1009F00BF04190C05165F
:108D600070206E286E2B000040080240022200296D
:108D7000016801D0114300E0914301607047C06871
:108D800080B270470246526800200A4200D001209B
:108D900070470000044A9068C90640094001C90EA6
:108DA00001439160704700000008024000B583B0A5
:108DB000002103200B46012201910090920203A1A1
:108DC000034807F0BDFA03B000BD0000434C490062
:108DD000D58D0001002498B0F4A725461594661E91
:108DE00038461294FFF75EFA81B2384602F058FD19
:108DF0000027FF433946684602F0EAFC0028F7D016
:108E00001598002805D000211591694609788142FE
:108E1000EED0129801281FD0022826D0684600788C
:108E20001B287DD009287CD00D287BD00A287AD039
:108E3000082879D07F2877D0014620395F29D7D2FA
:108E40003F2C72D2E5490855641CA4B20121684642
:108E500002F026FD2546CBE7684600785B2802D065
:108E600000201290C4E70220FBE700201290684621
:108E70000078412816D04228BAD1002EB8DB761EE1
:108E800057D4D7484078801BC01DC117490F091817
:108E9000C908C900401A8101D24809184038FFF7B3
:108EA0002DFA49E0CE48711C02789142A0DA407850
:108EB000761C801BC01DC117490F0918C908C900BD
:108EC000401A8101C74809184038FFF717FAC3480C
:108ED0000290FFF7E7F987B2C3A42046FFF7E2F953
:108EE00081B2204602F0DCFC0024002D0BD9C1A089
:108EF0000190FFF7D7F981B2019802F0D1FC641C10
:108F0000A4B2AC42F3D3B8A42046FFF7CBF981B2A8
:108F1000204602F0C5FC002F34D03946029805E007
:108F200036E038E0E2E0E3E029E136E102F0B8FCC7
:108F300028E0AA4900200870A8480290FFF7B2F97B
:108F400087B2A9A42046FFF7ADF981B2204602F00E
:108F5000A7FC0024002D0BD9A6A00190FFF7A2F9D1
:108F600081B2019802F09CFC641CA4B2AC42F3D321
:108F70009DA42046FFF796F981B2204602F090FCAE
:108F8000002FCAD13D469548FFF78CF984B22FE7F0
:108F9000012012902CE702F061FC904800252F463A
:108FA000019002F0F8FC1390224620210198FFF76F
:108FB0008EF9002860D10199085513991490002961
:108FC0005AD9149802F0EAFC224616900199FFF74C
:108FD0009EF9002819D1002F0AD102A81699FFF78F
:108FE0008DF902A8FFF75EF985B20DE06D1EADB2F6
:108FF000A54206D92A4602A81699FFF788F9002843
:10900000F4D1002002A948557F1C14981399401CE4
:1090100014908842D5D3002F64D0012F1AD0A542D6
:109020002BD902AF3F2C5DD2AC425BD23819012163
:1090300002F036FC0198395D0155641CA4B2F1E7D9
:109040003819012102F02CFC0198395D0155641C8E
:10905000A4B200E002AF3F2C44D2AC42F0D301985E
:1090600020210155641C63A5A4B22846FFF71AF914
:1090700081B2284602F014FC34E05FA52846FFF7D1
:1090800011F981B2284602F00BFC13980025002844
:109090001CD9284602F082FC074622460199FFF7B8
:1090A00036F900280ED13846FFF7FCF881B2384671
:1090B00002F0F6FB51A73846FFF7F4F881B23846C4
:1090C00002F0EEFB13986D1C8542E2D34AA52846B8
:1090D000FFF7E8F881B2284602F0E2FB214601984A
:1090E00002F0D8FC254602F0C9FB81E60A2000E028
:1090F0000D20159002F0B2FB3FA52846FFF7D2F8ED
:1091000081B2284602F0CCFB3449002008550D46B8
:10911000287800281FD0324C207800280AD06078A8
:10912000C01D4007C10D2F4808182946FFF7C1F898
:10913000002810D0607881012A4808182946FFF7D6
:10914000DDF86078401C4007400F607020780828E8
:1091500001D2401C2070002002F0D0FC1F4802F019
:1091600029FC1CA42046FFF79DF881B2204602F09E
:1091700097FB02F083FB002425463E4638E6002C90
:10918000B3D0641E1EA5A4B22846FFF78BF881B2A7
:10919000284602F085FB25462AE61AA73846FFF73F
:1091A00081F881B2384602F07BFB21E60D0A434C80
:1091B000492072656164792E205479706520276892
:1091C000656C702720666F7220636F6D6D616E64D1
:1091D000732E0D0A63616969632D3E00945000206F
:1091E00044470020D45000200D63616969632D3E1F
:1091F00000000000200000000D0A000020200000F8
:10920000082008000700000070B501F0C9FE044600
:1092100001F0C2FE05461B4A1BA11EA002F024FC61
:109220002348844203D123A002F06EFC08E00A2107
:109230002046FEF7BDFF0A46014626A002F014FCB8
:1092400001F072FF014629A002F00EFC2B48854276
:1092500003D12BA002F058FC03E0294630A002F015
:1092600003FC07F039F97D21C900FEF78BFF0146A9
:109270002FA002F0F9FB06F029FD014630A002F014
:10928000F3FB70BD0100010056312E30302E30311D
:10929000000000006669726D776172653A2025737F
:1092A000202830782530386C58290D0A000000003D
:1092B000FF7F0000636869702074656D703A20411B
:1092C000444320726561642074696D656F75740D27
:1092D0000A000000636869702074656D703A20258B
:1092E000642E256420430D0A000000007664643A71
:1092F000202575206D560D0A00000000FFFF0000BC
:1093000066616E2072706D3A206E2F6120286E6F3C
:1093100020746163686F6D65746572290D0A0000C1
:1093200066616E2072706D3A2025750D0A0000008E
:10933000757074696D653A20256C7520730D0A008F
:109340006672656520686561703A20257520420D5A
:109350000A00000070B50AA002F0D6FB0B4D0024F5
:1093600020460C21484341194A68295808A002F0B8
:109370007BFB641C052CF3D308A002F0C5FB70BD79
:10938000636F6D6D616E64733A0D0A00B013010175
:109390002020252D38732025730D0A006B65797305
:1093A0003A20544142203D20636F6D706C657465B6
:1093B0002C2055502F444F574E203D206869737420
:1093C0006F72790D0A00000070B50C46032823DB8C
:1093D00060680178312902D0322906D01CE040783B
:1093E000002819D1184E012504E04078002813D137
:1093F000164E402516A1A068FEF75BFF00280FD08F
:1094000014A1A068FEF755FF00280ED012A1A06895
:10941000FEF74FFF00280DD011A002F075FB70BDC4
:109420002946304600F0BEFA08E02946304600F0F2
:10943000B5FA03E02946304600F086FA11A0A2688A
:10944000616802F011FB70BD000C01400008014092
:109450006F6E00006F666600746F67676C65000072
:1094600075736167653A206C6564203C317C323EDF
:10947000203C6F6E7C6F66667C746F67676C653EC0
:109480000D0A00006C656420257320257320646F2D
:109490006E650D0A0000000010B507F01DF87D2173
:1094A0000446C900FEF76EFE0246214610A002F0F7
:1094B000DBFA06F001FA014614A002F0D5FA06F034
:1094C0000BFC044606F002FC024605212346090374
:1094D00011A002F0C9FA1DA002F016FB27490020D6
:1094E0000870084606F0D6FA244802F00DFB10BDBD
:1094F000757074696D653A20256C75207469636BAD
:10950000732028256C752073290D0A007461736B14
:10951000733A2025750D0A00686561703A20746FF2
:1095200074616C20257520422C20667265652025AB
:109530007520422C206D696E2065766572206672FA
:10954000656520257520420D0A0000006E616D657D
:109550002020202020202020202020202073746123
:10956000746520207072696F2020737461636B28AA
:10957000772920206E756D0D0A000000B44E002082
:1095800010B506A108A002F06FFA0DA002F0BCFA17
:109590001948016819A002F067FA10BD56312E3043
:1095A000302E3031000000006669726D776172659F
:1095B0002076657273696F6E3A2025730D0A00007C
:1095C0006D636D2D6464632D626C653A20424C4579
:1095D00028726474737329202B2046726565525477
:1095E0004F53202B205541525428444D4129202BC4
:1095F00020434C490D0A0000004000205379737449
:10960000656D436F7265436C6F636B203D20256C05
:109610007520487A0D0A00004860704701681A4AB0
:10962000114001600021016041608160C160174A02
:109630001749904204D148680F2210434860704790
:10964000144A904204D14868F022104348607047A1
:10965000114A904205D148680F2212021043486017
:1096600070470E4A904205D148680F2212031043FA
:10967000486070470A4A9042FBD148680F221204A2
:109680001043486070470000FEFF000008000240E1
:10969000000002401C000240300002404400024032
:1096A000580002400029016802D00122114301E064
:1096B000014A114001607047FEFF00000246096840
:1096C0000020114200D001207047000030B4036830
:1096D0000D4A0C6A13408A684D6922430C692C4379
:1096E00022438C692243CC6922434C6A22438C6A10
:1096F00022431A430260CA6842600A68826049686D
:10970000C16030BC704700000F80FFFF002B01D00C
:1097100010617047002010617047000001494861E6
:109720007047000000040140054B002219685B6986
:109730000140034202D0002900D0012210467047A8
:109740000004014010B4837919490268002B28D025
:109750000B6893430B604A6803689A434A60027936
:10976000521813680468234313608A6803689A4395
:109770008A60CA6803689A43CA604279102A06D090
:1097800051180A68006802430A6010BC70478A6872
:1097900003681A438A60CA6800680243CA6010BC42
:1097A00070470079401801689143016010BC704710
:1097B000000401400B680022002B56D0F0B40124B5
:1097C0000B68944023424AD04B68022B01D0122BE5
:1097D00016D113070AD5456A5307DB0E0F269E40A4
:1097E000B5434E699E402E43466209E0056A530721
:1097F000DB0E0F269E40B5434E699E402E43066207
:109800004B68012B05D0112B03D0022B01D0122B5A
:1098100006D14568DB06DB0FA54393402B4343602D
:109820000568530003279F400E79BD43B607B60F66
:109830009E402E430660C5688E68BD439E402E4301
:10984000C66085680126A543CC6894402C4384609B
:10985000C46A9E400D69B4439D402543C5620B68B0
:10986000521CD340ABD1F0BC704770470549016032
:10987000002242600F218260416101210261C160CA
:1098800070470000FF3F00008162704781617047B0
:1098900042694A404261704782B0EFF30884FEF7A4
:1098A00025FC400701D5EFF309840AA000F084FBF2
:1098B000E06800900CA0A3686268216800F07CFB5F
:1098C000E069009014A0A3696269216900F074FB4B
:1098D000FEE700000A2A2A2A204861726446617560
:1098E0006C74202A2A2A0A00523020203D25303864
:1098F0006C5820523120203D2530386C582052328F
:1099000020203D2530386C5820523320203D253012
:10991000386C580A00000000523132203D253038A2
:109920006C58204C5220203D2530386C5820504334
:1099300020203D2530386C5820785053523D25303A
:10994000386C580A0000000010B5FFF7A1FF10BDE9
:1099500030B505460E4887B00C46854202D101213C
:10996000042004E00B48854210D10121082000F0BA
:1099700021F90948844209D86846FFF777FF01209A
:109980000190694600942846FFF714FF07B030BDE8
:1099900000080140000C0140FF3F000010B5FFF738
:1099A00073FF10BD10B5FFF771FF10BD10B400219B
:1099B0004156FF23CAB29207D40E4278A3409207C1
:1099C000120EA24000290BDA0907090F08398C088A
:1099D0001049A4006118CC699C431443CC6107E092
:1099E0008C080D49A40061180C689C4314430C605A
:1099F000827801210078002A04D0C006C00E814080
:109A0000064803E0C006C00E81400548016010BC56
:109A10007047000000ED00E000E400E000E100E03D
:109A200080E100E0F7B5FFB004460025A5B00520B1
:109A3000EFF31087FF210090453102A8FEF727FCC5
:109A4000EFF31086FF21453153A8FEF720FC53A801
:109A5000013001909822224953A8FEF7FFFB012014
:109A600080F310880198804786F3108801221D49F1
:109A7000120303265300360388420AD194421AD0B7
:109A80009C4201D1151116E0B44210D101256D029E
:109A900011E0154988420AD1944201D115460AE0E5
:109AA0009C4201D11D4606E03546AC4203D00098E9
:109AB0007FB028B0F0BD06ACFF22013441320B4923
:109AC00002A8FEF7CBFB012080F310882846A69A57
:109AD000A599A04787F310887FB028B0F0BD00009B
:109AE00004090101C440130085601300C40701018B
:109AF00010B5EFF31084012181F31088FF210906CE
:109B0000401803490968884784F3108810BD000095
:109B10000440002010B5084806490160074941602B
:109B200007498160C922920006490748FEF796FB63
:109B300010BD0000B5480020044000204949002025
:109B40001D480020A80901011448002010B5EFF3BA
:109B50001084012383F31088FF231B06C018034BD6
:109B60005B68984784F3108810BD00000440002013
:109B7000034AD16A102399430143D1627047000020
:109B800000100240044A0029516901D0014300E05D
:109B9000814351617047000000100240044A0029CF
:109BA000916A01D0014300E0814391627047000057
:109BB00000100240044A0029916901D0014300E0ED
:109BC0008143916170470000001002400122054965
:109BD00012060128086802D09043086070471043BD
:109BE000FBE700000010024030B4164A516804231D
:109BF0001940154B01D0042901D0036001E013493D
:109C000001605168124B8906890F5B5C0168D9407D
:109C1000416053680F4C5B055B0FE35C0D46DD4014
:109C2000856053689B045B0FE35CD940C160D16AD7
:109C3000C90601D5084901E07D21C903016130BC95
:109C400070470000001002400090D0030048E80177
:109C50009C090101A009010100093D0070470000B5
:109C600010B5FEF759FA044606F03CFC002803D074
:109C700001200349000748602046FEF751FA10BD55
:109C800000ED00E010B50A4C2069411C01D000280D
:109C90000AD10120064934220003FFF7C3FE2069E0
:109CA000411C03D0002801D0024810BD002010BD87
:109CB000E047002009480020F0B5564C85B0E06927
:109CC00021040843E0618120534D00062863534876
:109CD0006861534828625348032201689203914304
:109CE0000160514934228014FFF79CFE4E4B4F4EC9
:109CF00018694F4F411C29D0002827D0A9691A782C
:109D000049094901D206D20E0A43AA612168EA1321
:109D10009143216021687F2212029143000208438F
:109D200020606068304360606068B843606060686D
:109D3000211508436060206A3E4908402062206A7D
:109D4000D96809020843206205B0F0BD6168204669
:109D5000314361606168B943616061680127BF0296
:109D600039436160002104917D21C90003910021E4
:109D700000917F2140240025029501910268610233
:109D80008A4302600E11234908687F221202904321
:109D9000220202430A600520FEF7A0F90120FEF727
:109DA0009DF91C48406B800704D4284603996D1C1C
:109DB0008842F3D91748C06B80B2B04201D9811BE9
:109DC00000E0311AB94202D2E2B28FB20292B0423E
:109DD00001D3019400E00094019A00988018C00516
:109DE000000EA04203D0044604988142CBD8094813
:109DF00001687F2212029143029A12020A43026012
:109E0000416849084900416041684907FCD405B0F0
:109E1000F0BD000000100240007000400F0800007C
:109E20001800020000100140E0470020000001007F
:109E300000070000FF00F8FF10B50A4C2069411C24
:109E400001D000280AD10120064934220003FFF77F
:109E5000E9FD2069411C03D0002801D0014810BD54
:109E6000002010BDE047002010B501F0CDFC10BD72
:109E700010B40B06CC065B0FE40E0121A140012BB0
:109E800007D0022B07D01430002A026805D00A43FD
:109E900004E00C30F8E71030F6E78A43026010BCAB
:109EA000704700000029818903D001225203114329
:109EB00001E0024A1140818170470000FFDF00008D
:109EC000002A828A01D00A4300E08A4382827047D6
:109ED0000246128800200A4200D00120704770B468
:109EE0000A06530FCE060125F60E2A460024B2407C
:109EF000012B0FD0022B10D0838A1340090A00884F
:109F00008D402840002B02D0002800D0012420469C
:109F100070BC704783891340F0E7038AEDE70000C7
:109F200070B50446008A86B00D461B490840E98892
:109F300001432182A08919492A890840A98811432F
:109F40006A8902431143A181A08A15490840A98961
:109F50000143A1826846FFF747FE1248844201D1BF
:109F6000039800E002982968192289005043FEF7FF
:109F700009F906466421FEF705F90501280964215F
:109F80004843301A00013230FEF7FCF80007000F9A
:109F90002843208106B070BDFFCF0000F3E9000028
:109FA000FFFC0000003801408088C005C00D7047EC
:109FB000C905C90D818070470FB410B503A9044BC2
:109FC000044A029800F004F910BC08BC04B0184719
:109FD00009BF0001C40100200FB410B504A9074B4C
:109FE00002AA039800F0F4F8044602A9002000F049
:109FF00096FC204610BC08BC04B018471FA90001FD
:10A000007CB51546024600201C4600290BD0491E8F
:10A0100000920191044B6A462146284600F0D8F888
:10A02000009A002111707CBD09A900012021020CB9
:10A0300001D010211046020A01D010460839020949
:10A0400001D01046091F820801D01046891E42081F
:10A0500001D0881E7047081A70470000F0B51FB481
:10A0600086B00998089A030D0021024314D0514884
:10A07000514A1818504305141198012810981AD005
:10A08000281A401C00264D4F4D490096019104901E
:10A09000002812DA444211E01198012449A3012852
:10A0A00001D11098C1430698119A84600360C26080
:10A0B00041600BB0F0BD4042E4E7044621050020BA
:10A0C0003F4A001C51410391029012E0E00707D083
:10A0D00032463B4601990098FEF770FA01910090D4
:10A0E00032463B4610461946FEF768FA06460F46CA
:10A0F0006410002CEAD10498039B0028029A099965
:10A10000089806DAFEF75AFA019B009AFEF756FA0B
:10A1100005E0FEF7BBFA019B009AFEF7B7FA04468A
:10A120000E460022284BFEF78BFC03D80020C043CC
:10A13000014607E00022254B20463146FEF78CF908
:10A14000FEF75AFB102409E0002C0ADB0A22002348
:10A15000FEF742F8079B30321A55641E02460A4346
:10A16000F2D11122641C079B121B1C19119B012B9D
:10A1700003D0012308430ED10AE0084304D0112084
:10A1800010900020119077E71098151A6D1E0BE0C3
:10A190001098824202DD00236D1C03E0824201DA46
:10A1A00000236D1E002BEED0069811998260C160CD
:10A1B00030C07EE701FCFFFF104D0000000014409E
:10A1C0000000F03F300000000000F0430000E03FDE
:10A1D000FFB597B00646002518E2252877D1002460
:10A1E0002746FD49049400E00443761C32780120A0
:10A1F000203A90400842F7D130782A280ED0022227
:10A20000307801463039092916D804990A23594370
:10A21000303940181443761C0490F1E7189802C8AE
:10A2200004911890002904DA0120400304434842B5
:10A23000049002200443761C30782E2814D1042088
:10A2400004437078761C2A2809D11898761C80C897
:10A25000189009E00A214F43303FC719761C307827
:10A26000014630390929F5D930786C2810D006DC40
:10A270004C281AD068280ED06A2817D104E0742818
:10A2800013D07A2812D110E00120400504430CE0DD
:10A290000121090501E0032109050C437178814280
:10A2A00003D1012000052418761C761C307811900B
:10A2B00066280BD013DC58287DD009DC00287BD021
:10A2C0004528F6D04628F4D047281AD1A5E118E051
:10A2D000632835D0642870D0652812D19DE170289C
:10A2E0006CD008DC6728F1D069287BD06E280DD0AF
:10A2F0006F2806D1BAE073282ED0752871D078283F
:10A3000059D01A9A199990476D1C7EE16002400F4E
:10A31000022809D003280DD00428189801680DD010
:10A320000D60001D189070E11898EA1701680D6023
:10A330004A60F6E7189801680D80F2E70D70F0E7C3
:10A3400018986A4601781172001D1890002050720A
:10A3500002A80090012005E0189802C8189000207B
:10A360000091C04361070DD5002101E00199491C0E
:10A370000191B94212DA8142F8DB009A515C00295E
:10A38000F4D10BE0002101E00199491C01918142C7
:10A39000FADB019A0099895C0029F5D101990498AA
:10A3A0001A9B471A21463846199A00F097FA0199E4
:10A3B000401945180BE04FE02CE113E04EE0009807
:10A3C00000990078491C00911A9A199990470198B0
:10A3D000401E0190401CF2D1214638461A9B199A22
:10A3E00010E137E00A200021009001916002410F46
:10A3F000022907D0189A01CA1892C2179446032955
:10A4000008D00AE01898C01DC108C90005C91891F4
:10A41000944607E000B2C2179446042902D140B224
:10A42000C1178C4600226146944506DA0A4600218F
:10A43000404291418C462D2102E0210504D52B217B
:10A440006A461173012103E0E10701D02021F7E7FB
:10A45000029155E00A200AE0102008E01020009048
:10A460000021042004430191082703E00820002173
:10A47000019100906002410F022907D0189A01CA89
:10A48000189200229446032908D008E01898C01DAD
:10A49000C108C90005C91891944603E080B2042997
:10A4A00000D1C0B200210291210729D5119970294C
:10A4B00006D0009A1021019B4A401A4305D00EE0B5
:10A4C00040216A461173012108E06146014306D02C
:10A4D00030216A4611731199517302210291009A39
:10A4E0000821019B4A401A430AD16146014301D128
:10A4F000610705D530216A46117301217F1E029143
:10A500001199582904D035A10E910DA90D910DE096
:10A5100037A1F9E76146019B009AFDF75DFE0E9BAE
:10A520008C469B5C0D9A521E0D921370614601433E
:10A53000F0D10D9805A9081A20300190600703D5C5
:10A5400001200004844300E001270198874201DDD7
:10A55000381A00E00020019900904118029809186B
:10A560000498401A0490E00306D421461A9B199AD5
:10A57000049800F0B3F94519002706E003A81A9AD9
:10A58000C05D199990476D1C7F1C02988742F5DBCE
:10A59000E0030CD521461A9B199A049800F09EF905
:10A5A000451904E01A9A3020199990476D1C0099BA
:10A5B000481E00900029F5DC08E00D980D99007800
:10A5C000491C0D911A9A199990476D1C0199481EC2
:10A5D00001900029F1DC63E10928010030313233B8
:10A5E00034353637383961626364656600000000CF
:10A5F00030313233343536373839414243444546B9
:10A600000000000000F05AF94519761C3078002847
:10A6100000D0E2E528461BB0F0BD600700D4062755
:10A620001898C01DC108C90048680A680831C30FDE
:10A63000DB071891190001D09CA108E0210501D584
:10A640009BA104E0E10701D09AA100E09AA1430098
:10A6500011985B08109165280CD006DC452809D0BC
:10A6600046281DD0472841D141E0662818D06728E8
:10A670003CD13CE00021112F01DB112000E0781CCF
:10A680000191009008A911A8FFF7E8FC1399059122
:10A690000021119A15927F1C12980197009150E0A9
:10A6A0000120C00703900120019008A9009711A87C
:10A6B000FFF7D4FC139A149905920022119B009283
:10A6C00012981593059A0192002901D0104602E0D4
:10A6D000791C40180190381A01D5019804E04042D5
:10A6E000401E0090781C0190C01B029043E0012F97
:10A6F00000DA01270021112F01DD112000E038468A
:10A700000191009008A911A8FFF7A8FC13990591E1
:10A71000119A0021129815920091019721070CD4EB
:10A720000599B94201DB019900E00191012904DD9D
:10A73000159A491E515C302906D0B84201DA011D34
:10A7400005DA0121029115E00199491EEDE7002883
:10A7500005DC0099411800910199091A03E0019A5A
:10A76000411C914200DD01910099401A401C029069
:10A770000120C0070390200706D402990198814266
:10A7800002DB0020C043029000206946C87707AF73
:10A79000012103980337C907884224D00220119071
:10A7A0002B201290039800280CDA404203902D20B1
:10A7B000129007E00A210398FDF7E4FC30317F1E78
:10A7C000039039701199481E11900029F2DC03980A
:10A7D0000028EFD1791E12980870307820210840A7
:10A7E0004530BF1E387006A8C01BC01D03901098CE
:10A7F0000078002800D00120019941180298C01764
:10A800000918039809180498401A401E0490E003A0
:10A8100006D421461A9B199A049800F05FF845194E
:10A8200010980078002803D01A9A199990476D1C47
:10A83000E00324D521461A9B199A049800F04EF89B
:10A8400045191CE00098002807DB0099059888420C
:10A8500003DD1598405C199901E0199930201A9A86
:10A86000904700986D1C401C00900298401E02907A
:10A87000002804D11A9A2E20199990476D1C01992D
:10A88000481E01900029DDDC05E038781A9A7F1C0B
:10A89000199990476D1C0399481E03900029F4DC18
:10A8A00021461A9B199A0498ACE600002D0000007E
:10A8B0002B0000002000000000000000F8B5044656
:10A8C00000251E461746880404D405E0394620209A
:10A8D000B0476D1C641EF9D52846F8BDFFB5044687
:10A8E000002581B01E46C80301D5302700E020278F
:10A8F000880404D505E038460399B0476D1C641EF2
:10A90000F9D5284605B0F0BD4A68002A06D00A6885
:10A91000531C0B6010704868401E486070470A68FE
:10A92000531C0B601070704700B599B060216846E9
:10A93000FDF7ADFC042008AAD07012A000680190B9
:10A940000B2010AAD070024610A109A8FDF786FCC2
:10A95000002010AA107101215171D0719171907372
:10A960001175D082A02010839176B4209083192095
:10A97000C001D08308480090684602F019FF19B062
:10A9800000BD000003160A18000000000AFFFFFFC8
:10A990004E6174696F6E73009DA9000170470000DD
:10A9A00010B58CB000240094019402940394049494
:10A9B000059406940794089409940A94FFF762F9A1
:10A9C000002804D0014601A8FEF790F807E012A085
:10A9D00001886A4691804188D180808810816946CB
:10A9E000CC704C810A20887012220A7303A80CA133
:10A9F0000130FDF733FC0C20694608841820488498
:10AA0000FF208C84F530C8840A480885684602F027
:10AA100091FF0CB010BD0000010203040506000008
:10AA200043414949432D4D434D2D32303236303963
:10AA3000303200008813000000B583B00D4900914A
:10AA40000D4900200191029069460872684603F0A2
:10AA500075F8FFF7A5FF00F059F9FFF765FF074804
:10AA600002F012FE064802F00FFE02F0C5FE03B02F
:10AA700000BD000085AA00015DB5000139AE0001EE
:10AA800045B30001017801291AD070B500250D4E9B
:10AA90000D4C02290BD0032908D102F0ADFE00F0C5
:10AAA0001FF840213046FEF779FF257070BD402128
:10AAB0003046FEF777FF2570F72002F0EDFF70BDFE
:10AAC000704700000008014037470020034800217C
:10AAD0000170418081804170704700004C47002028
:10AAE00010B5044800210170418000F0D7FD00F04E
:10AAF0008FFB10BD4C470020F3B583B004980024B1
:10AB000000286ED954480090544A03981178005D8B
:10AB1000002904D001290BD002291AD122E0CA2829
:10AB20007ED14F490870012050800521918017E0A7
:10AB30004B4B51885854491C88B2508005286FD11E
:10AB40000098417803780802FF211843E1318842D8
:10AB500003D900201070508076E0C01D9080022044
:10AB6000107071E03D4A3E4B51885854491C88B2E0
:10AB700050809188884267D10098002241780078FF
:10AB80000D02054337488446E81C86B23648002E3D
:10AB900014D9364F6146895C0902484000210304FC
:10ABA00002D54000784000E04000491CC9B280B2A4
:10ABB0000829F4D3521C92B2B242EBD328494A1965
:10ABC000937956791A023243904239D148788F7876
:10ABD000491D11282AD005DC012808D010282FD1C2
:10ABE00024E037E0122821D0202829D124E00126B2
:10ABF0003F2D10D82A461E48FDF730FB1C49002087
:10AC000048551C4800F07AFF194800F0D3FE06466C
:10AC1000002000F073FF68460671012301AA00E0DE
:10AC200012E03946032000F027F809E00A462B46D7
:10AC3000394600F0F9FA03E02A46384600F0D4F924
:10AC40000649002008704880641C0498A4B284421D
:10AC500000D259E705B0F0BD175500204C47002041
:10AC60001455002015550020FFFF000021100000A2
:10AC7000D4540020D9EB0001F8B51C461346024617
:10AC8000E01D80B20090FB2802D90020C043F8BD2F
:10AC90001A4DCA2028706A70A970200AEC702871B9
:10ACA000002C04D022461946681DFDF7D7FAE01C97
:10ACB00085B2134F13480022002D13D9124EB95CF0
:10ACC000090248400021030402D54000704000E022
:10ACD0004000491CC9B280B20829F4D3521C92B278
:10ACE000AA42ECD3054909194871000A8871034842
:10ACF000009900F0DBFC0020F8BD00001457002094
:10AD000015570020FFFF00002110000000B587B09C
:10AD1000002001900090039004906A460690107302
:10AD20000C49029105219170032313701023D370F5
:10AD30005070107101235371907150730648059043
:10AD40007D20917300011082104603F0BDFB07B017
:10AD500000BD000040E2010000B0030110B5024850
:10AD600003F05AF9002010BD284E00202F4800792A
:10AD700000285AD1F8B56D202C2303220721400169
:10AD80000CF4DAD6A0210446017029480027C178C6
:10AD9000617027710321E1806772012666710721C6
:10ADA000244D2177A9796177687B002803D0E7805B
:10ADB000032060710EE0E87900280BD0A879022802
:10ADC00000D166772671E6802046A979203041704F
:10ADD0008670077015488079022804D0032815D0A2
:10ADE00004281BD116E003F061FB00280BD00520DE
:10ADF000E0806771688A6061688AA06120460A30D5
:10AE000003F082F90AE0094903208871288B606108
:10AE1000288B02E0E88B6061E88BA0610348067133
:10AE2000467120460CF4C4D6F8BD7047844D00200E
:10AE3000084E0020744E002010B584B00A2303226F
:10AE4000072110480CF478D61B21017000214170B5
:10AE50001424448003228280C1800B4A02810CF4B6
:10AE6000A7D66846048009480190684602F02EFE85
:10AE7000684604810648039002A803F00BFE04B064
:10AE800010BD00001B0D0000FF010000DC120101DD
:10AE90006DBC0001FFB585B0054602A800901C46B8
:10AEA0002846069903F05AFB6846007A002866D0C7
:10AEB00006980090280A334A019403900E2826D061
:10AEC000314800240178002951D92F48E1000818A1
:10AED000828803998A4240D1009A81689646019AF5
:10AEE000284694460A791206120E36D00968254B78
:10AEF000D700083FCE1937887668BFB2874201D0A5
:10AF00009F4226D1634603227146B04725E01F4980
:10AF1000681809282BD800981D49844608792E46C0
:10AF200000062346000E1ED0C4000F68083C3C19E2
:10AF300027886468BFB2B74201D0974204D1032288
:10AF400061462846A0470EE0401E0006000EEBD1E9
:10AF500009E0521E1206120ECAD10B48641C00787A
:10AF6000E4B2A042B1D86846007A002807D0094868
:10AF7000426C002A02D0284606999047002009B06A
:10AF8000F0BD0000FFFF0000304D0020EEF1FFFF9C
:10AF90002C0E0101844D002000487047FFFF000087
:10AFA00070B50E4D01212846FDF7E0FE702002F03D
:10AFB000EDF8044600212846FDF7D8FE08498C42EA
:10AFC00001D1481070BD2046FDF706FE0549FDF78A
:10AFD00006FAFDF7F7FB00B270BD00000008024062
:10AFE000FFFF000000002041F7B5002090B015469B
:10AFF0000E46002A04D0012D04D13178FF2901D159
:10B00000444E06250024002D7BD904A90746039150
:10B01000305D0E9007286FD20100794409794918F4
:10B020008F446A030E32354C5C003B480F9004207D
:10B0300000900FAB39460E9A039802F0F9F85CE0E5
:10B0400001213648FDF792FE702002F09FF8009033
:10B0500000213248FDF78AFE31490098884201D12B
:10B06000401007E0FDF7B8FD2E49FDF7B8F9FDF7F0
:10B07000A9FB00B269460881022202AB3946009260
:10B08000039802F0D5F838E0FFF786FF0BE0602068
:10B0900002F07CF82249884201D1002003E06021BF
:10B0A000FDF7C4FD80B2694688800220009001ABA4
:10B0B00039460E9A039802F0BBF81EE005F00CFA30
:10B0C0007D21C900FDF75EF80F90042000900FABC2
:10B0D00039460E9A039802F0ABF80EE004F0F6FD44
:10B0E0000F90042000900FAB39460E9A039802F09F
:10B0F0009FF802E005E0FFE73846641CA4B2AC42CA
:10B1000083D3034604AA21201099FFF7B5FD13B09D
:10B11000F0BD0000EC130101010001000008024035
:10B12000FFFF00000000204110B5602002F02EF863
:10B130000449884201D1002010BD6021FDF776FD51
:10B1400080B210BDFFFF000010B502F02BFF0448D5
:10B150000169002901D004208847002010BD0000AB
:10B16000944E002070B5224C606B224DC00722D057
:10B17000A06B21497E2209685143401A2988491E43
:10B1800029804B21C90040181C49884213D3002054
:10B190002880206A4008400020621949086802049B
:10B1A000930F184A01D0904300E0104308601648FE
:10B1B000407F02F02FFC298801200029216B07D055
:10B1C000014321630522032110480CF477D70DE0D9
:10B1D000FF22120291432163216B05229202114347
:10B1E0002163216B0143216303F0AEF9002070BDA0
:10B1F00000100240344700208C000020B104000001
:10B200000010014000C00000E44D0020010F0000CC
:10B2100004480021017041618161C1610162816264
:10B220007047000054470020F8B514460D4610281A
:10B2300009D0112878D0122804D11A462146284670
:10B2400003F09CFAF8BD00910C2B04D000230122DE
:10B250001021284664E02278E178104662780906D9
:10B2600012021043A2781204104308430502E0784A
:10B270002D0A00062279054310466279E17912020F
:10B280001043A27909061204104308430602E0792C
:10B29000360A00060643082021180A7810464A7824
:10B2A000120210438A78C978120410430906084331
:10B2B0000702E07A3F0A000607431E481E49412460
:10B2C000A404884202D0A0420BD10C461B49281F7F
:10B2D00088420DD3002303221021009803F024FBA1
:10B2E000F8BD002302221021009803F01DFBF8BDD9
:10B2F00013484078002804D1FEF70CFC10490120C7
:10B3000048700F4801210170002141618161C161D4
:10B3100001628162001DF0C00B460A4610210098B0
:10B3200003F002FBF8BDFFE71A462146284603F06A
:10B3300079F9F8BD0080000100800001FD7F030065
:10B340005447002010B584B014230322072112486B
:10B350000CF4F2D31B21017000214170472444807A
:10B3600003228280C1800D4AC2600D4A0261072219
:10B3700002720CF41DD4684604800A4801906846A5
:10B3800002F0A4FB684604810748039002A803F07A
:10B3900081FB04B010BD00001B0D0000FC12010178
:10B3A000EC120101E412010145F300010020704795
:10B3B000F8B5184D184FE879002801D02E7B00E031
:10B3C000FE780322331D072114480CF4B5D3A921BC
:10B3D000044601701248C178617000216180E879EB
:10B3E0001049002803D02A7B896C201D02E0FA78DE
:10B3F000201D091DFCF732FF608802218019608042
:10B4000007480279062A00D00171417120460CF4E8
:10B41000CFD3F8BD744E0020544E0020A60D00007E
:10B42000844D0020344E0020F8B51F26232303222C
:10B43000072128480CF480D30446AA20264F207008
:10B44000F878264D6070E8786080EA782449201DFD
:10B45000FCF704FF6288B01AC1B2201D1018214AFF
:10B460000326032910D92B79002B0DD00670192340
:10B4700043705389091F1B0AC370937A83706388D2
:10B48000C9B21B1D6380001D02291AD96B79002BDC
:10B4900017D0137B891E8B4200D21946CDB2691C8E
:10B4A0000170117BA94201D1092100E008214170FE
:10B4B0002A460D49801CFCF7D1FE6088AD1C40195E
:10B4C00060803879062800D03E717E7120460CF4E9
:10B4D0006FD3F8BDA60D0000844D0020744E0020EF
:10B4E000584E0020084E0020154E002070B53A231B
:10B4F0000322072116480CF41FD3A421154D04463E
:10B500000170E8786070A97913480022022910D0F0
:10B51000032913D0042916D062802271807901F0AA
:10B52000ABFE052028710420687120460CF440D33E
:10B5300070BD018A642359436180EEE7C18A6423A8
:10B5400059436180E9E7818B642359436180E4E7D3
:10B55000A10D0000844D0020744E002070470000B3
:10B56000FFB50F4683B00021009101911646694650
:10B57000FDF7C2FA040030D10521C9026846FDF783
:10B58000C1FA002828D121496846FDF7BBFA0028F6
:10B5900022D11F496846FDF7B5FA00281CD11D4984
:10B5A0006846FDF7AFFA002816D12921090268463E
:10B5B000FDF7A8FA00280FD117496846FDF7A2FA4F
:10B5C000002809D115496846FDF79CFA002803D1E7
:10B5D00000988088C10B03D00624204607B0F0BD38
:10B5E00000050099000D0D186888B04200D20724AC
:10B5F0002988B819884201D90D24EEE7A8193A46DE
:10B60000001D0699FCF72AFE6F80E6E7012800007E
:10B61000032800000228000002290000032900007E
:10B620001FF4BED600F00EF8012004F013FAF7E77D
:10B6300010B503490020087000F004F810BD0000A8
:10B640004647002012480021007800281FD070B51E
:10B65000104D86B02878002817D1A8886C88A042A1
:10B6600013D00D4E6A4680B2A04209D0335C5354C9
:10B67000401CC005491CC00D89B2A8801429F2D312
:10B6800001202870104603F061FE06B070BD7047BF
:10B690003747002046470020D452002002490020AE
:10B6A000488088800870704746470020F0B4844680
:10B6B0000D480078002814D00022002911D90B4829
:10B6C0000B4D878843881C465B1CDB05DB0DBB42AA
:10B6D00007D06646B65C521C2E5592B243808A4211
:10B6E000F0D3F0BC704700003747002046470020E9
:10B6F000D452002030B58DB001210820FEF75AFA4F
:10B7000001218803FEF756FA02A8FEF7AFF84020A1
:10B7100002900220284D0424039002A90794284691
:10B72000FEF748F880210794029102A92846FEF707
:10B7300041F8E12040020890002069468884C884CE
:10B74000088588850C2048851C4D08A92846FEF7E9
:10B75000E7FB01210846FEF715FA194C2046FDF7D4
:10B760005DFF0123224617490220FDF7CFFF01228A
:10B7700080212846FEF7A4FB00220121402004F08E
:10B78000EBFA114C2060012004F0D4FA6060012231
:10B790000E492846FEF76CFB1C2069460870032002
:10B7A0004870012088706846FEF700F9012128469C
:10B7B000FEF778FB0DB030BD000C014000380140B1
:10B7C0000800024000000240384700202505000024
:10B7D00070B505460B480468002C0ED0481C0ED0EE
:10B7E00008467D21C9004843FCF7CCFC02462946A7
:10B7F000204604F018FC012800D0002070BD002075
:10B80000C043F3E73847002010B582B00020104C49
:10B8100000900E492046FEF762FB002814D0204617
:10B82000FEF7C2FB694608710A480068002804D088
:10B830000A46002301A904F0AFFB0098002803D0BA
:10B84000012005490007486002B010BD2505000031
:10B85000003801403847002000ED00E010B5064CEC
:10B860006068002807D004F027FE022803D1C11E1B
:10B87000606804F079FC10BD3847002010B5074C13
:10B880006068002809D004F017FE022805D10023C3
:10B890001A461946606804F0B8FA10BD384700200F
:10B8A00000283FD000293DD0F0B51F4E0C4605467C
:10B8B0008BB000213046FDF7F5FE1C4F02203946C3
:10B8C000FDF7AAFE1A480090102002900020802167
:10B8D00005910490032101950394090306900790B4
:10B8E000089009910A9069463046FDF7EFFE012164
:10B8F0003046FDF7D7FE39460220FDF7DFFE00286F
:10B90000F9D000213046FDF7CDFE39460220FDF783
:10B9100083FE084C40212046FEF7DAFA0028F9D0D1
:10B920000BB0F0BD7047000008000240000002406C
:10B930000438014000380140002230B4D243491E8F
:10B940000FD3094C03785A400023401C5508D207F6
:10B9500000D022465B1C6A40DBB2082BF6D3491E9E
:10B96000F0D230BCD04370472083B8ED02468B88BC
:10B970000020022B01D00D207047C988002A05D075
:10B980000029F9D00129F7D0812070470029FCD087
:10B990000229F9D17047052070470000052804D21C
:10B9A0000C214843024908587047002070470000A6
:10B9B000B013010170B588B000246A46234616E032
:10B9C000401C01782029FBD00929F9D00906090E6D
:10B9D00012D0A1005050641C00E0401C01780029E6
:10B9E0000AD0202901D00929F7D10370401C017821
:10B9F000002901D0082CE4DB002C14D0104E0025C7
:10BA000028460C21484331580098FCF752FC002886
:10BA10000CD06D1C052DF3D30AA0009900F024F87A
:10BA2000012008B070BD002008B070BD0C20454357
:10BA3000A8198268694620469047002008B070BD6A
:10BA4000B0130101756E6B6E6F776E20636F6D6D55
:10BA5000616E643A20257320287472792027686506
:10BA60006C7027290D0A00000FB410B503AB6021DC
:10BA70000648029AFEF7C4FA05490020C877034831
:10BA800000F042F810BC08BC04B018473450002045
:10BA900074500020F3B581B00D460198FCF702FC0C
:10BAA000144C86B22046FCF7FDFB81B22046FFF71E
:10BAB000F7FE0024002D0BD90F4F3846FCF7F2FBA0
:10BAC00081B23846FFF7ECFE641CA4B2AC42F3D35B
:10BAD000084C2046FCF7E6FB81B22046FFF7E0FE6B
:10BAE000002E03D031460198FFF7DAFE304603B04E
:10BAF000F0BD0000E8910001F491000101490860E7
:10BB0000704700004047002010B507490968002928
:10BB100001D0884710BD0446FCF7C4FB81B2204623
:10BB2000FFF7BEFE10BD0000404700200246002087
:10BB3000802901D98D207047062A06D0072A07D010
:10BB4000082AF8D10729F5D170470829F2D17047A2
:10BB50000629EFD370477047704770B5C468054633
:10BB60006068002803D00020002802D00CE00120EB
:10BB7000FAE7201DFCF7CCFF0BF4CED66068002856
:10BB800008D000200028F4D00020E86020460BF404
:10BB9000C3D670BD0120F5E730B40446A289092060
:10BBA000521C93B2E48900222546D540ED0707D008
:10BBB0005D1C8D4202D130BC104670479B1C9BB26D
:10BBC000521CD2B2092AEFD330BC7047FFB585B002
:10BBD0000E9D04462F8801201E4600213A46CA4089
:10BBE000D20704D04B0003225B1C9A401043491C2F
:10BBF000C9B20929F2D3049030461E210840218A97
:10BC0000184A00230191009302920390132304AA7F
:10BC100015490698FCF782FF009000281FD10121EA
:10BC200014200BF403D70746E06006980188B98119
:10BC30002988F981F00701D00120C0030799084342
:10BC40003880208A788014206082204600F060F8D6
:10BC5000381DFCF769FF208A00210CF43DD00098C4
:10BC600009B0F0BDEC0C01010A1800000048704753
:10BC7000840D0101FFB5087881B00C46092836D241
:10BC8000142002F0D3FE0746217800F0EFF80028D8
:10BC90002BD061782078FFF749FF060028D17D6816
:10BCA000002D0ED020782979814207D12946381DF0
:10BCB000FCF740FF28460BF42FD602E02D68002D3C
:10BCC000F1D16078012108300BF4B0D60546207818
:10BCD0002871607868716278A11CA81DFCF7BEFA13
:10BCE0002946381DFCF72CFF02E0822600E0812661
:10BCF00002230648039A04990BF41ED72178017099
:10BD000046700BF455D7002005B0F0BD01140000BB
:10BD100010B50446142002F089FE04492160032175
:10BD20006181123060600120208110BD940D0101FD
:10BD3000F8B517460C4610460BF4BCD7012831D194
:10BD4000142002F073FE0546017C00F08FF80646D1
:10BD5000297C22781448914214D1697C63780902C5
:10BD60003A46891D9B1D0BF4E7D605460680002048
:10BD70002871607868806278A11C681DFCF76EFAF3
:10BD8000284609E0697C062309023A46891D0BF41E
:10BD9000D3D60680802101710BF40AD700213846E2
:10BDA0000BF49AD70020F8BD140C0000F8B50F462C
:10BDB000002409781846254609291DD20B007B442A
:10BDC0001B79DB189F440407101313130A160D0088
:10BDD000052414A510E00A2414A50DE0082416A5D6
:10BDE0000AE0072417A507E00A2418A504E00524A3
:10BDF00019A501E006241AA50146A31C1A480BF454
:10BE00009BD60646387830707470002C04D02246D9
:10BE10002946B01CFCF722FA30460BF4C9D60020A4
:10BE2000F8BD00004E53494E470000004E532D42CE
:10BE30004C452D312E300000123456FFFE9ABCDEE8
:10BE400000000000025E044000000300312E302E8E
:10BE5000302E302D4C450000312E302E30000000A9
:10BE6000FFEEDDCCBBAA00000314000010B48289F1
:10BE7000C489521C93B200222046D040C00706D08D
:10BE8000914202D15B1C9BB205E09B1C9BB2521CF1
:10BE900052B2092AF0DB092A02D010BC18467047BA
:10BEA00010BC00207047000070B5050005D0134E8F
:10BEB0003068854203D1002070BD72B6FEE703F002
:10BEC00081FD6C6903F08AFD7068844202D0B0681D
:10BED000844201D1022070BD0948844204D1A86A7D
:10BEE0000028F7D1032070BD0648844203D0002CFF
:10BEF00001D0012070BD042070BD000084470020E7
:10BF0000EC580020D858002070B50D4D04460A2882
:10BF100009D10D212846FEF74BF880212846FDF770
:10BF2000D7FF0028F9D0E1B22846FEF741F880217A
:10BF30002846FDF7CDFF0028F9D0204670BD00004F
:10BF400000380140F0B50878324F334D334E801E33
:10BF500083B00C46062859D2010079440979491862
:10BF60008F4402255434543A01203070A07868760A
:10BF7000A078C00705D02A492A48FCF7B7FD387ACF
:10BF8000A874B28A002A06D0FF20F5307080032101
:10BF900025480CF493D0F169002937D00020009097
:10BFA000019005206A461070684688472EE00024FC
:10BFB0006C7601F0A9FCF169002927D000940620D5
:10BFC0006A4601941070684688471FE01722A11C3A
:10BFD0001648FCF743F919E0B8780001C019403061
:10BFE000807D002812D11C22A11C1148FCF736F9D3
:10BFF0000F48A18A0182E18A4182218B8182618B73
:10C00000C1820B49608A0883207F6874002003B0D6
:10C01000F0BD0000844D0020C84C0020E44C0020FE
:10C020008D4D0020DB4C0020040F0000C24C00208E
:10C03000A84C0020F0B518460D46014685B02223D5
:10C04000032274480BF478D5012104464170287806
:10C050000B286ED201007944097949188F4405CD27
:10C06000CDCD6F6ABB23CDCD6C00012020706070F8
:10C070006948817921710179A170C1796171417932
:10C08000E170017AA171417AE171817A2172C1690D
:10C0900000294ED00020009002206A4610706846A9
:10C0A00001948847A9E0072020700120607068464D
:10C0B0001FF4D4D2019F009EFCF7BEF88019608265
:10C0C0000025FCF7B9F88119601900908170FCF720
:10C0D000B3F8C11900986D1CEDB20175082DF0D3AD
:10C0E0000825FCF7A9F8B919401861196D1CEDB2C3
:10C0F0008870102DF5D310202077484881780901E9
:10C1000008184030807D012877D11C22A11C4448AA
:10C11000FCF7A4F84248A18A0182E18A4182218B7E
:10C120008182618BC1823E49608A08833D48217FBC
:10C13000417462E0052000E00A2020705DE00422E6
:10C1400022706878012804D0002802D0022833D059
:10C1500053E00120304D6070287C002810D002A8E8
:10C160001FF47CD2FCF768F82F49FCF70BF82F4836
:10C170000818029940182E49FCF704F8009101E0D4
:10C18000E8680090E969002907D0002002900320A8
:10C190006A46107202A8039288471021A01CFCF77F
:10C1A00076F80098A0700098000AE0700098010CE2
:10C1B0002171000E607120E01748C169002905D087
:10C1C00000200090019068460270884720460C3895
:10C1D0000BF4E4D414E00620164D2070E878012812
:10C1E00011D01021A01CFCF752F8A9886182E988BF
:10C1F000A1822989E1820020207620460BF4D8D440
:10C20000002005B0F0BD10220B49A01CFCF726F859
:10C21000EBE70000140E0000E44C0020844D0020E9
:10C22000A84C0020C84C0020A0BB0D00A086010037
:10C230003F420F00084E0020934D002000B50848F3
:10C2400083B0026C002A08D00020009002900520E4
:10C250006B461870684601919047002003B000BDFE
:10C26000844D002010B584B0FF2B19D0144C226CE3
:10C27000002A08D000200090029006206B4618701B
:10C2800068460191904703200BF414D5032814D17C
:10C29000A26F002A11D003210A480BF40FD70CE03B
:10C2A00009480123007F03220102084808310BF4EA
:10C2B00043D4072101700BF47BD4002004B010BDDF
:10C2C000844D0020090E0000E44D0020050E000002
:10C2D000FFB5180A4C4E83B00C46B070FF287DD0D5
:10C2E000010234230322494808310BF425D40546C2
:10C2F000B07800270101891940318872B07821880F
:10C300000001801940300181B078617A0001801904
:10C310004030C172B07862890001811940318A8150
:10C32000A289CA81E0890882207C012802D00028E5
:10C3300007D00BE0B17801200901891940318875D7
:10C3400004E0B07800018019403087752088308083
:10C35000607A307221460A312D48FCF7C7FB02F0A3
:10C36000A5F800281BD0607A012804D103221146C9
:10C3700028480BF431D402F0A1F805280FD20100AF
:10C380007944097949188F440606060206000120FF
:10C390002821485505E005212820415501E02820A5
:10C3A0004755032105980BF497D417203086B178B0
:10C3B00009018919403148821748C068002803D014
:10C3C000032116480BF4DAD51548028D002A03D054
:10C3D000032114480BF472D6306C00E00EE0002804
:10C3E00008D0022069460097087002950194316CCC
:10C3F0006846884728460BF4DBD301E001F0FCF9DE
:10C40000002007B0F0BD0000844D0020020E0000A7
:10C410008D4D0020150D0000944E0020030F0000EC
:10C42000084E0020020F000030B5180A144D00011C
:10C430000C46401983B0FF214030817201F0B0FA00
:10C44000002803D1022103200BF446D42A6C002AD1
:10C4500008D00020009002900320694608706846CA
:10C460000194904710210748FBF711FF0648006828
:10C47000002802D009200BF419D2002003B030BDEF
:10C48000844D0020A34D0020100C002000B508486A
:10C4900083B0C169002907D00020009001900920D5
:10C4A0006A46107068468847002003B000BD00004F
:10C4B000E44C0020FFB591B00D46122303224348FF
:10C4C00014990BF439D300210446017040480078D8
:10C4D000002862D03E48407C002833D03C2168468A
:10C4E000FBF7D5FE01F0D4FD002841D004A90F913F
:10C4F0003749461EF0B23A228969504341186846CE
:10C50000091DFBF7ABFE6846008B2988884206D1DF
:10C510000822A91C0F98FBF7E4FE00280BD0207816
:10C5200000280BD008A8407C607410226946601C6B
:10C53000FBF794FE1CE001202070F3E73006000EAC
:10C54000D6D12AE023482988008B884225D10822A9
:10C55000A91C2148FBF7C5FE002809D10120207045
:10C560001E481022407C60741A49601CFBF776FE5E
:10C570002078002811D01648C169002907D0002072
:10C580000090019007206A46107068468847204650
:10C590000BF40ED3002015B0F0BD0D48C169002981
:10C5A00007D000200090019008206A46107068466D
:10C5B0008847022303220A4814990BF4BDD20121B3
:10C5C0000170062141700BF4F3D2E0E7180E000071
:10C5D000E44C0020A84C0020B84C0020C84C00209F
:10C5E000040E000070B50C4609781B481B4D1E4612
:10C5F000002904D0012912D002292BD11AE01C23D2
:10C6000031460BF499D2064620783070287B708032
:10C610002A7B1349301DFBF721FE304607E00A2331
:10C6200031460BF489D221780170698941800BF47D
:10C63000BFD20FE00A2331460BF47ED2217801707D
:10C64000298C4180698C8180A98CC180E98C018111
:10C650000BF4AED2002070BD0B0E0000084E00207F
:10C66000154E002010B5087800F006FE002010BD21
:10C6700005480A8842861A0A1201101809884030B3
:10C680008182002070470000844D002030B5180AD8
:10C69000C043000683B00D46000E21D0190A0902DE
:10C6A000E12006230322000108310BF445D20446A1
:10C6B0000120207002206080FF204130A0800B48C4
:10C6C000026C002A08D000200090042069460870FF
:10C6D000684601950294904720460BF469D201E028
:10C6E00001F08AF8002003B030BD0000844D002026
:10C6F00000B5084883B0026C002A08D000200090E2
:10C70000029008206B4618706846019190470020FF
:10C7100003B000BD844D002070B518460C4601469C
:10C7200002230A480BF408D205460949A078087389
:10C730006288211D0748FBF791FD00206870207872
:10C74000287028460BF434D2002070BD0D0E000076
:10C75000084E0020154E00204A780B48002A05D0CC
:10C760002030012A08D0022A09D00AE00279012AE1
:10C7700007D10978C17004E00978017501E00978F2
:10C780004175002070470000844D002070B5487846
:10C79000002806D0FF25124C01280BD0022816D005
:10C7A0001BE010480179062917D10721017100F01B
:10C7B00091FF12E0207DFF280FD001F089F80A4890
:10C7C00025750169002908D00020884705E0607DB3
:10C7D000FF2802D001F05EF86575002070BD0000F2
:10C7E000A44D0020844D0020944E002010B5032B52
:10C7F00006D010220548891DFBF730FD002010BD32
:10C800000348017A034801F0F9FCF7E7A34D002043
:10C81000844D00208D4D0020F0B50D460878E34E84
:10C82000E14934464978002720348DB0A1287AD0D8
:10C8300012DCDF490C911B2876D006DC012819D0C8
:10C8400003287CD017286DD14FE128286ED091287D
:10C850006DD0A02866D152E10246A23A092A61D2DF
:10C8600013007B441B79DB189F44FE5CFDFD5CFDDF
:10C87000FCFDFD006878002854D1012002F03AF94F
:10C8800001F0FAFC342303220721CA480BF454D1E7
:10C8900003210170C84904468A7842700122C27699
:10C8A000FB224284C54AC284C54A82840A88028423
:10C8B00087768A888280CA88C2800A892281487ADB
:10C8C0008009032805D188780522104201D1012072
:10C8D000A076A07E04221043A076BA486080C87873
:10C8E000012825D0204610210A30FBF7D0FC316CFE
:10C8F000002907D001206A4600971070684601950C
:10C9000002948847012000F0B7FC20460BF450D178
:10C91000012303220721AC480BF40ED11A21017028
:10C920000BF446D133E11EE1CAE008E069E049E0DA
:10C93000204610220A300C99FBF790FCD7E70097AD
:10C94000019702970397049705970697079708970B
:10C9500009970A970B9701F0A9FD002805D06846B2
:10C9600001F0EAFB0AA801F0B7FB01F09FFD0028E7
:10C970000CD068468079002808D108A8807B002860
:10C9800004D00121684601F01DF800E18A4C694697
:10C99000A0880880E0884880208988808F711022D4
:10C9A00002A80C99FBF75AFCE078012804D00697FE
:10C9B000079708970997E4E7102206A80C99FBF758
:10C9C0004DFCDEE7E07B002813D111230322072171
:10C9D0007E480BF4B1D00546282028707648C078F0
:10C9E000012808D01021681CFBF751FC28460BF4E5
:10C9F000DFD0E773CBE01022681C0C99FBF72EFC0C
:10CA0000F4E7012002F076F8012103200BF464D151
:10CA10006F48012444841F20049067480178490628
:10CA200001D57F21049181780522114204D0FF2293
:10CA300004998132114304910088C00504D5032173
:10CA40000498490208430490082162480191029029
:10CA500003210B2304AA00970394C9025E48FCF744
:10CA60005DF802E079E04AE089E0002846D15B48C1
:10CA700006218786FF2005905948019102900823DE
:10CA800005AA0097039457495748FCF747F8002830
:10CA90007DD100F009FE002879D1022103200BF49A
:10CAA0001BD1B079012808D000F0CEFE3E48407876
:10CAB000C0076CD001F010FA69E000F09DFE66E05E
:10CAC00001F0F4FCE77300F0EFFD00285FD10221D4
:10CAD00003200BF401D1B0790128EED000F0B4FEB0
:10CAE00031484078C007E5D151E0687800284ED041
:10CAF000F179481EF0713D4801F050FB47E0717933
:10CB0000491E052906D8A72802D13079002806D168
:10CB100000F0E0FD2878A42801D0A72837D170794B
:10CB2000042806D0062804D0082808D00C282ED1C6
:10CB30000CE02F480168002929D0B07904E01A4898
:10CB40000169002923D00120884720E016480169A7
:10CB500000291CD00320884719E03771FF20F070AE
:10CB60002075607513E0207DFF2802D068780028CA
:10CB700002D000F0ADFE0AE0C8079BD107E0607D5F
:10CB8000FF2802D06878002804D000F083FE00203F
:10CB90000DB0F0BDA07D0028F9D08807F7D5E17D64
:10CBA000144801F007F9F2E7944E0020844D00206C
:10CBB000934D0020040D0000084E002005020000E7
:10CBC00048080000A08C0000190D0000230D000093
:10CBD000B00B002068110101D20B0020680B00206F
:10CBE000C0110101011800009C0B00208D4D002098
:10CBF000344E0020BC4D002070B500250C46284660
:10CC0000401C0628FCDB254E2246307E31461A3277
:10CC1000C96906282AD203007B441B79DB189F448C
:10CC200024020910171E0622A01CFBF75AFB00283D
:10CC30001BD01BE0237E092000F05CFF002814D1EC
:10CC400014E0237E212000F055FF00280DD10DE0D7
:10CC5000237E162000F04EFF002806D106E0237E3A
:10CC6000192000F047FF002800D001250C48807DE6
:10CC7000002811D17169002901D020468847002D74
:10CC80000AD03169002901D00220884701F0A6F9B5
:10CC9000217AA01C01F08EF8002070BD944E002077
:10CCA000A44D002010B50A78000A000210434A780B
:10CCB000FF231B02120298431A4010438A781B027A
:10CCC000120498431A401043C9780002000A09066A
:10CCD0000843FBF7BAFA002010BD10B510460AF45D
:10CCE000E9D7002010BD0020401C0628FCDB0020F6
:10CCF00070470000F8B51C4617460D4610460AF46A
:10CD0000D9D7002811D1472001F090FE0646042310
:10CD10003A46032106480AF40FD7210A01702988F0
:10CD2000B288891A41800AF443D70020F8BD000078
:10CD30000D470000F8B517460C46472001F076FE77
:10CD400021780646122901D013291BD1B068054667
:10CD50000C351229C288018916D006230F480AF41F
:10CD6000EBD669884180617801710AF421D7B068F7
:10CD7000002803D00AF4D0D50020B0600021384646
:10CD80000AF4AAD70020F8BD042305480AF4D4D633
:10CD90006988018061788170E7E700000947000039
:10CDA0000747000000B5084883B0026C002A08D08D
:10CDB00000200090029009206B461870684601918F
:10CDC0009047002003B000BD844D002030B5104DC9
:10CDD00083B0088828861C0A200140190A88403040
:10CDE00042822A6C0025002A07D0009507206B4656
:10CDF000029518706846019190470648A100405876
:10CE0000002801D04030C574002003B030BD0000C0
:10CE1000844D0020580B0020FFB581B00020009009
:10CE20000E4603980AF446D7002802D001284CD0B9
:10CE30004DE0142001F0FAFD07463188FEF7ACFE04
:10CE400005462448092D36D27C68002C1ED0217955
:10CE5000A94203D02468002CF9D117E0002C15D08A
:10CE60006379039A9B1D04990AF466D605463088B7
:10CE7000288000202871607968806279A11D681D72
:10CE8000FBF7ECF928460AF493D620E03D740498A9
:10CE9000010A7974384601F0C1FD014601230E48AC
:10CEA000039A0AF449D605700AF482D60121039840
:10CEB0000AF412D70BE00623039A04990AF43CD62D
:10CEC0003188018080210171DDE702200090009807
:10CED00005B0F0BD140C000002140000FFB585B0D1
:10CEE0000E4607980AF4E6D6002802D0022009B0C0
:10CEF000F0BD472001F09AFD0290002069460870BD
:10CF00000898070A308802F06AF900246946054645
:10CF10008C8000281ED102981622016A684600788B
:10CF200003465043024610328A5A5204920F1FD1D0
:10CF30000A5C401C085C1E4900021018884217D188
:10CF400002AA03A9184602F05DF802986946C05D7E
:10CF500088800224A31D1748079A08990AF4ECD583
:10CF60000746308838803D717C80002D15D019E04F
:10CF70003946029801F052FD014604230E48079AF3
:10CF80000AF4DAD507706946097841800AF410D6A8
:10CF9000012107980AF4A0D607E0224601A9781DCE
:10CFA000FBF75CF938460AF403D6002009B0F0BD5F
:10CFB00002290000140C000004470000FFB58BB0EC
:10CFC0000C46472001F032FD0025694605900D749E
:10CFD0000E9804A9070A208802F001F9060061D121
:10CFE00005981622016A6846007C504302461032BA
:10CFF0008A5A5204920F3AD10A5C401C085C3049AC
:10D0000000021018884232D102950395208800F062
:10D0100093F802A9002300911A4608A9FBF796FD90
:10D020006846008C012109030840C043C004C017B2
:10D030002146401CFEF79AFC0606360E32D16846A1
:10D040000997007C0190A57907AA694601F0DAFFEB
:10D050006846028806A80799FBF700F906A909980F
:10D060000A460D5468460188019802F009F83946CD
:10D07000059801F0D3FCA1880D9A891D8BB2014659
:10D0800010480AF459D50546A288A11D801DFBF75A
:10D09000E5F82F706846007C6880A088A880284644
:10D0A0000AF486D5042308480D9A0E990AF444D54B
:10D0B0002188018086700AF47BD500200FB0F0BD76
:10D0C000022900000A470000160C0000F0B589B0E4
:10D0D0000446FBF741FD05460026154F1BE006A957
:10D0E0002046FBF709FD002302AA01A906A8009625
:10D0F000FBF738FD68460089B84203D169460979D3
:10D10000022911D00B49884203D1684600790228D0
:10D1100007D0641CA4B2A888A04202D8E888A04224
:10D12000DDD2002009B0F0BD204609B0F0BD0000FE
:10D130000229000003280000F0B589B00446FBF77F
:10D140000BFD05460026104F14E006A92046FBF70C
:10D15000D3FC002302AA01A906A80096FBF702FD52
:10D1600068460089B84203D1641CA0B209B0F0BD82
:10D17000641EA4B2A888A04202D8E888A042E4D2E3
:10D18000002009B0F0BD000003280000F8B5254DCF
:10D1900007462878224C244E002816D10121080386
:10D1A000FCF7F0FC0020FCF7E3FC0120FCF70EFD8F
:10D1B0003046FBF77FFD03213046FBF7EBFD0121F5
:10D1C0003046FBF7ABFD0120287039463546304626
:10D1D000FBF7FBFC01212846FBF796FD01212846C1
:10D1E000FBF7D0FD002807D1641E13D0012128468B
:10D1F000FBF7C8FD0028F7D001212846FBF7E2FC29
:10D200002846FBF7BCFD044600212846FBF77CFDC1
:10D210002046F8BD00212846FBF776FD0348F8BDFF
:10D22000A08601008047002000080240FFFF0000A8
:10D2300030B4029C42540546491C88B22C54401C10
:10D24000002180B2002C07D95A5C2A54401C491C8A
:10D25000C9B280B2A142F7D330BC7047054CFF255C
:10D26000F53501212046FCF76FFB284602F0F2FB62
:10D27000F7E70000000C014010B5A023094902287F
:10D2800009D0002203280AD0042808D00B704A7065
:10D2900000F0A2F810BD0B7080204870F8E7E02085
:10D2A0000870F4E711400020F8B52A4920204860B2
:10D2B00029480121C163294905228A610021C163EE
:10D2C00027490B20086100F087F82748254A0263A8
:10D2D00026494163264B8363264CC4632748264D69
:10D2E0000560274E4660274981602749C16027496C
:10D2F0000161274941612749816127490163284824
:10D3000026494160274FC760274F07610262274ABD
:10D3100042628362C46205634663254A8263254A8A
:10D32000C2632648244A0260184A4260244A826046
:10D330000163244981632448244A41688918244AA6
:10D34000914206D2234982680A63C2684A6300692F
:10D350008863F8BD00100140C0270240402502400C
:10D36000402702400259F80040280240025B850035
:10D37000025A8000025D8500025F805080280240D2
:10D3800002000878020A0800026EAC500259FC0044
:10D390000200C8001270131402700314026E2800F9
:10D3A000C0280240025D0500125B0500025B84009C
:10D3B000020A0600026E2C5002C3BF000029024080
:10D3C0001200AC00125D0500104000206F2895FF90
:10D3D000AF590F00C026024030B415481549037DEF
:10D3E000154AFF2B06D1407DFF2803D11348407812
:10D3F000C0070CD01248134B04789C604078D86169
:10D4000011480861114B8B62106030BC7047104BA3
:10D410000B6110484861104C8C61104D8D62C862E0
:10D420000F48086313600F485060946030BC704729
:10D43000A44D00200028024040280240944E0020C5
:10D440001140002000270240127E0200127E0300DD
:10D45000027E020002C2A00012C70000027E03008A
:10D4600012C7800002C2E00082B021491F48086351
:10D47000FEF740F91FA0FCF79FFD29A0FCF79CFDDB
:10D4800030A133A0FCF798FD3748016837A0FCF7BE
:10D4900093FD3DA141A0FCF78FFD49A0FCF78CFD59
:10D4A000FDF7CAFAFDF712FB01215048FCF750FACC
:10D4B00040214F48FCF74CFA01F03AF802200024D2
:10D4C0000202009023464BA101944B4802F038FF22
:10D4D000012000900023802248A10194484802F0D6
:10D4E0002FFFFBF763FC02F08FFBFEE7008000815B
:10D4F000007000400A3D3D3D3D3D3D3D3D3D3D3DD3
:10D500003D3D3D3D3D3D3D3D3D3D3D3D3D3D3D3D4B
:10D510003D3D3D3D3D3D3D3D3D3D3D3D3D0A0000E8
:10D52000206D636D2D6464632D626C653A20424CFE
:10D5300045202B204672656552544F53202B2043C3
:10D540004C490A0056312E30302E30310000000098
:10D55000204669726D776172652076657273696FB6
:10D560006E2025730A0000000040002020537973CC
:10D5700074656D436F7265436C6F636B203D20254E
:10D580006C7520487A0A000043414949432D4D43B8
:10D590004D2D3230323630393032000020424C4589
:10D5A00020656E61626C65642C20616476657274BE
:10D5B0006973696E6720617320222573220A000057
:10D5C0003D3D3D3D3D3D3D3D3D3D3D3D3D3D3D3D8B
:10D5D0003D3D3D3D3D3D3D3D3D3D3D3D3D3D3D3D7B
:10D5E0003D3D3D3D3D3D3D3D0A000000000C0140FC
:10D5F00000080140424C450021B600014C45440062
:10D600005DD2000110B50124E4022046FCF78CF83D
:10D61000002805D02046FCF781F80D49022008704B
:10D62000012424032046FCF77FF800280AD0204676
:10D63000FCF774F8BFF34F8F07490648C860BFF383
:10D640004F8FFEE705484068002800D0804710BD96
:10D65000800000200400FA0500ED00E040400020BA
:10D6600006480068002800D08047BFF34F8F054967
:10D670000348C860BFF34F8FFEE700004040002022
:10D680000400FA0500ED00E0064A11780A2907D2E5
:10D690008900891848601078401C1070012070477C
:10D6A00000207047044D002010B5084C084AE1796D
:10D6B00013780020994207D288008018406880477C
:10D6C000E079401CE071012010BD0000844D002075
:10D6D000044D0020F8B5324D052629792846807979
:10D6E000304C08290CD20A007A44127992189744D7
:10D6F00003080D1313191C2A052801D0FDF736FB6A
:10D70000F8BD022808D0FDF753FEF8BD607B002865
:10D7100002D1E079002802D0FDF7E8FEF8BDFDF760
:10D7200083FEF8BD06202871F8BD022303220721DD
:10D730001D480AF401D2A5210170E9784170072142
:10D7400029716E7128E002230322072117480AF489
:10D75000F3D10746A7203870E97879700620687100
:10D760000020287103200AF4A5D2032812D0A8793A
:10D77000012804D0022802D003280BD104E0207D28
:10D78000002801D0032003E0A07E002802D004205E
:10D79000A87100E0AE7138460AF40AD2F8BD000064
:10D7A000844D0020744E0020A20D0000A30D000047
:10D7B00010B5002804D0014660220C48FAF74EFD4F
:10D7C0000B490C48CA781C2A04D9427B002A01D193
:10D7D0001C22CA70C1781F2901D91F21C170017B89
:10D7E000E22901D9E221017310BD0000344E00206E
:10D7F000544E0020744E0020114901220879072858
:10D800000CD08879002809D0012801D0052806D13C
:10D810000C48827B002A03D002200CE08A717047FA
:10D82000027D002A01D0032005E0807E002801D07F
:10D83000042000E00520887110B5FDF797FA10BDAF
:10D84000844D0020744E002070B5104C0525A07941
:10D85000062809D201007944097949188F44020247
:10D8600004040403A57170BDA571022303220721DE
:10D8700007480AF461D1A5210170E17841700721C0
:10D88000217165710AF494D170BD0000844D0020AF
:10D89000A20D000010B50B4C607DFF2810D00223B4
:10D8A0000322072108480AF447D1A7210170617DAE
:10D8B0004170064A00215171FF2161750AF478D147
:10D8C00010BD0000A44D0020A30D0000844D0020D9
:10D8D00010B50A4C207DFF280ED002230322072119
:10D8E00007480AF429D1A7210170217D4170054A1A
:10D8F000002151710AF45CD110BD0000A44D00203C
:10D90000A30D0000844D002010B508480223807844
:10D9100003220102064808310AF40ED101210170E8
:10D92000132141700AF444D110BD0000844D002041
:10D93000040E000010B584B0002804D001462A224D
:10D940000E48FAF78BFC0EA00FC86C460FC40B4BA9
:10D95000002069461C180A5C247922430A54401CA2
:10D96000C0B20628F6D310220A48FAF777FC0A4913
:10D970000A48FBF7BBF804B010BD0000084E0020B9
:10D98000501921901F04D5624FA489AB90D0CF23AA
:10D9900000000000934D00200C4E0020FC000020F1
:10D9A0000020074B01460A01D2184032927AFF2A22
:10D9B00001D0401CC0B2491CC9B20329F3D370473F
:10D9C000844D0020F8B507460B46282043430D46FA
:10D9D000032207210E489B1C0AF4AED0912101704E
:10D9E000002406464570002D0ED9204628214843C4
:10D9F000C1190022CA7180192822801CFAF72EFC56
:10DA0000641CE4B2AC42F0D330460AF4D1D0F8BD85
:10DA1000910D0000F8B57D262025F600184B194C15
:10DA20001949032812D00A6A01273A430A620A6A8E
:10DA30009207FCD50A6AAA430A6201281AD0022872
:10DA40001AD01E60FBF794F82060F8BD0F480F272E
:10DA500082683F023A438260086A042210430862E7
:10DA6000086A0007FCD5086A284308623D200001C7
:10DA70001E60E9E7064800E006481860E2E700009B
:10DA80008C00002090000020001002400010014097
:10DA9000D10300005704000010B5044608480423D1
:10DAA0008078032201020748891D0AF445D00649FF
:10DAB0004C8001210170002141800AF479D010BD11
:10DAC000844D0020010C0000F00B0020084A117862
:10DAD0000A290AD2C9004368891800688B60486027
:10DAE0001078401C10700120704700207047000023
:10DAF000304D0020FFB581B01C00064618D01078CC
:10DB0000411CA14214D8032C12D3401EC5B2507838
:10DB1000971CB04206D12A4638460299FAF7E1FB33
:10DB2000002808D07A19601B801E0406240EE6D156
:10DB3000002005B0F0BD012005B0F0BDF0B50446F1
:10DB40006F4E704883B06D4FB168C1626E4901631A
:10DB5000F16A8162F16B4163B16B816331467C2272
:10DB600040313846FAF77AFB00257D60FD607D6222
:10DB70006648B8627D64BD64FD643D666448B8660D
:10DB80006448386264486549057003200870644839
:10DB9000F91401600904016089140160F0686149A9
:10DBA0000746401E0088604B884200D01F60366EDA
:10DBB000701E0088884200D05E6001200003009043
:10DBC000694601950D710820487101278F716846DB
:10DBD000FBF7B8FD84215548FAF759FB2A21544830
:10DBE000FAF755FB60215348FAF751FB52484F4969
:10DBF000056145618561C561056245628562C562F1
:10DC0000FF264E48CE700675467500200201521858
:10DC10004032401CC0B296720328F7D320680864D3
:10DC20006068486446486189C187217A454803296C
:10DC300001D8417700E0457701212020FBF7A2FFC2
:10DC4000414A4249042000F083FE424940480860AE
:10DC50000A464149052000F07BFE404A4049072022
:10DC600000F076FE40493F4808600A463F490820D8
:10DC700000F06EFE3E4A3F49092000F069FE3E4832
:10DC800005633E48414907703D4805703D480570B1
:10DC90003D48086001203E49C00208803D494F20B0
:10DCA00008703D49082008703C48072106704670FE
:10DCB0008670C170057145718571C571114838490B
:10DCC000C1613849016238494162002001F0D6FC47
:10DCD000364903200AF444D00021032009F4FCD77C
:10DCE000002000F007FF012303220721304809F438
:10DCF00023D7077009F45CD703B0F0BDC00900203A
:10DD000000800001C000002061D600010D47002006
:10DD100095F7000105D60001C6000020D8000020BC
:10DD200000E100E0FEE7000040400020844D0020BC
:10DD3000084E0020344E0020844E0020A44D0020C8
:10DD4000C44D0020E44D0020804000208080010070
:10DD5000350E0101C0400020C080010000410020BC
:10DD600000DB0100814100204041002040DB010038
:10DD7000C0460020C061020000700040600000202A
:10DD8000C9000020610000200090D0036C0000203A
:10DD900068000020630000206400002008010020CB
:10DDA00095E90001BDEA00015DEA0001C812010128
:10DDB000020D0000F8B5404D0646687D3F4C0F4609
:10DDC000FF281CD02046C268002A03D003213C480B
:10DDD0000AF474D13A23032207213A4809F4ACD655
:10DDE000A4210170697D0446417037480022017802
:10DDF00000291ED00121A170A28002701BE06D20BD
:10DE0000022303220721400109F496D6A2210170C2
:10DE10002E49C978417009F4CBD6EF7531462C48AC
:10DE2000FAF764FE0120A87560780221084360704B
:10DE3000F8BDA270A2800120E07019214901E180A3
:10DE400022482181038CE381438C2382838C63826B
:10DE5000C38CA382FF23E2824133184D23836D7864
:10DE60006D070DD50525E5706181A181018CE184E7
:10DE7000418C2185818C6185C08CA085E2852386BB
:10DE800038200755204631463230FAF72FFEE07829
:10DE9000810703D50220FFF7EFF906E0400701D51F
:10DEA000032000E00120FFF7E7F90A490C20487140
:10DEB000204609F47DD6F8BDA44D0020944E0020E4
:10DEC000030F0000A10D0000044E0020084E0020AA
:10DED000BC4D0020844D0020F8B52C4E2C4D317DDA
:10DEE00001276878FF2941D0C1073ED0B843687048
:10DEF0002849002008703A2303220721264809F404
:10DF00001BD60446A4202070307D60702878A07055
:10DF100068788006800F20716888E080A88820815A
:10DF2000E888E08128892082E7700120FFF7A4F9C2
:10DF3000687840070AD5E07802210843E0706888D5
:10DF40006081A888A0810320FFF796F96878000710
:10DF500003D5E0780C210843E0701049082048718F
:10DF60000020B075204609F423D6F8BD3843687008
:10DF70006D20022303220721400109F4DDD5A121F0
:10DF800001700749C9784170EDE70000A44D0020F9
:10DF9000944E0020044E0020A10D0000844D00206E
:10DFA000084E002010B50A4C607DFF280ED00223D9
:10DFB00003220721074809F4BFD5A5210170617D1F
:10DFC0004170054A0D21517109F4F2D510BD0000D0
:10DFD000A44D0020A20D0000844D002070B50B4C14
:10DFE000207DFF2811D00A4D687909280DD0022321
:10DFF00003220721074809F49FD5A5210170217D3F
:10E0000041700921697109F4D3D570BDA44D002078
:10E01000844D0020A20D000010B504464088A18860
:10E020000246491C19234A43DB019A420FDC0628A9
:10E030000DD3228890420AD3E2887D23DB009A42E6
:10E0400005D84B00C9184843D100884201DD0020A3
:10E0500010BD0D480E238078032201020B480831C1
:10E0600009F46AD509210170218841806188818085
:10E07000A188C180E188018100214181491E8181FF
:10E0800009F496D5012010BD844D00200E0E00002D
:10E0900010B5084A084B906901888478994206D1E6
:10E0A000917CA14204D20024FBF722FD00E0002471
:10E0B000204610BDE44C0020341200000B4610B581
:10E0C00004493A228969504341181846091DFAF754
:10E0D000C5F810BDE44C002010B590B004463C21BA
:10E0E0006846FAF7D4F8FFF7D3FF401EC0B269467E
:10E0F000FFF7E4FF08A8807CA0710CA9204603313B
:10E10000FAF7F4FC10B010BD10B590B004463C21F5
:10E110006846FAF7BCF8FFF7BBFF401EC0B269467D
:10E12000FFF7CCFF08A8007CA0710AA920460231A5
:10E13000FAF7DCFC10B010BD10B590B004463C21DD
:10E140006846FAF7A4F8FFF7A3FF401EC0B269467D
:10E15000FFF7B4FF0AA920460231FAF7C7FC08A866
:10E16000007CA071204606A9102208300231FAF77F
:10E1700075F80848C17820461830012904D01021CC
:10E18000FAF785F810B010BD10220349FAF766F8C7
:10E1900010B010BD084E0020934D002070B590B017
:10E1A0000D460646FFF774FF002D23D0854221D887
:10E1B000182303220721104809F4BED4044617206F
:10E1C0002070012060703146A01CFAF78FFC3C21C2
:10E1D0006846FAF75CF86D1EE8B26946FFF76EFF15
:10E1E000204606A9102208300231FAF737F82046F7
:10E1F00009F4DED410B070BD140D0000F3B58FB07B
:10E200000C463C216846FAF742F8FFF741FF012C23
:10E210001AD0002816D0154D0AAE0236441EE0B2C0
:10E220003A22A969504341186846091DFAF716F8C1
:10E23000062231460F98FAF754F800280DD0200630
:10E24000000EEBD111B0F0BD0949421ECA71014662
:10E250000F98FFF7A3FF11B0F0BD06A910220548E3
:10E260000231F9F7FBFF11B0F0BD0000E44C0020D3
:10E27000844D0020A34D002070B5284C82B020684A
:10E280008003FCD5264D687FFFF7C4FB606A606A97
:10E29000012630436062606AB04360622148C08FEB
:10E2A0000A2811D9E16932071143E1611E494A6820
:10E2B00032434A601E491D4A0A6003224A60886050
:10E2C0001C4808601C48086068461DF4C7D11B49FB
:10E2D00000980860687FFF252D02032811D000F008
:10E2E00027F9206BA8432063206B3F214902084394
:10E2F0002063206B3043206301220321104809F47E
:10E30000DDD610480168A94301600F490868FF2263
:10E3100012049043086002B070BD0000001002407B
:10E32000E44D0020C44D002040100240555500002F
:10E3300000300040AAAA0000CCCC000048400020D9
:10E34000010F000000E400E008E400E0F0B5D7B001
:10E3500054A81DF483D14A490024886AC96A549993
:10E360000122411A09010909D206914204D954999E
:10E37000081A000100094142424E40290CDC708815
:10E38000002809D0401E7080142203213E4809F461
:10E3900095D6002057B0F0BD3C48FF21569029315A
:10E3A0006846F9F774FF707CB569002832D0FFF732
:10E3B0006FFE69468870B17C6F4688420BD23A2165
:10E3C00048430246291D381DF9F748FF69468878F9
:10E3D000401C887008E03A21401E48430246294606
:10E3E0003E31381DF9F73AFF694688783A214843AB
:10E3F000C0190A4636385699F9F730FF244869465D
:10E400000880B069FBF774FBFF2227326946B069C8
:10E41000FBF79CFBFF20F53070804A944B944C94A2
:10E420004D944E944F945094519452941748539451
:10E43000418D40AA1185818D5185C08D9085154CE7
:10E4400048AA257C9573102213494CA8F9F706FFBA
:10E450001248C078012804D11022114950A8F9F7B8
:10E46000FDFE01260F48002DC67306D1A07C0028B2
:10E4700003D001214AA8FFF7A5FA0B48067088E7E8
:10E48000C0800240E44C0020040F0000A84C002093
:10E4900034120000C84C0020C24C0020084E00205E
:10E4A000934D0020A44D0020044E00200248007827
:10E4B000002800D001207047E44C0020014800797A
:10E4C00070470000E44C002070B517493CC80E4668
:10E4D00084B040363CC64368026880684B65134C84
:10E4E0000A658865607C002818D0002569460D7291
:10E4F000FBF710FBFFF7CCFD69460872E1690126C6
:10E50000002906D068460095067002A8019068466A
:10E5100088476846007A002802D0267004B070BD93
:10E52000257004B070BD0000A84C0020E44C002011
:10E5300004490868401C0860012801D00120704788
:10E54000002070472440002003490868002802D0BA
:10E55000401E08600120704724400020F8B50C469A
:10E560002849294B4118294F294A0026069D002990
:10E5700008D0012922D0274940180A282FD301208A
:10E580002870F8BD20780A2838D22149800009581F
:10E59000214A914203D11E490E501E502EE0B9422D
:10E5A0002CD10322082311461C4809F4C5D2217836
:10E5B00001706168416009F4FBD21FE020780A28ED
:10E5C0001CD280001158B94218D119581150207826
:10E5D000134962684018032109F470D50EE0C0B2F7
:10E5E0000A280BD284001159002907D0B94205D05E
:10E5F000094FB94202D016511E5188472E70002093
:10E60000F8BD0000FBF0FFFF804C00208FF80001F8
:10E61000584C0020F9F0FFFF8DF80001060F0000B4
:10E62000070F0000F7B5534F3878002809D0042AA7
:10E6300009D2012211217B69009800F075F903B01D
:10E64000F0BD002314E00C784E7820468C7836021A
:10E65000CB783043240420431B061843CB780002B8
:10E66000000A1B0618437B690D1D141F984206D033
:10E6700002221121009800F057F903B0F0BDB868EC
:10E680001E19864203D90322112100986DE07E6194
:10E69000F869B0420FD2F96978684018FBF728FA98
:10E6A000002801D0052207E00120F96900030818BD
:10E6B000F861B042EFD30022002A3CD1B86A0028AA
:10E6C00022D02D49042808D2002C1BD02B780B54C3
:10E6D000401C641E6D1CB862F4E73E46042811D14C
:10E6E000B1697068244B401804221946FBF72EFAD2
:10E6F000002801D0052203E0B069001D0022B061AE
:10E700000020B062002A16D1042C1DD3BA697868A3
:10E71000A608B600801829463246FBF717FA0028EB
:10E7200001D0052203E0B86980190022B861AD1953
:10E73000A41B002A08D011217B69009800F0F4F88E
:10E74000FCF766FD03B0F0BD002C05D0224629463B
:10E750000948F9F783FDBC62BB693A6A0098190B56
:10E760009142EFD939620022112100F0DDF803B0A7
:10E77000F0BD00005447002078470020F7B5634DF6
:10E780008CB028780B46002809D0042A09D0012231
:10E7900012216B690C9800F0C7F80FB0F0BD002390
:10E7A00013E01A78D97810465A78090612021043F5
:10E7B0009A781204104308430402D878240A000609
:10E7C00004436B69A868834206D0022212210C9888
:10E7D00000F0AAF80FB0F0BDA86A0026002815D0F6
:10E7E000042806D24A4AFF211154401CA86204287A
:10E7F000FAD3AB69686846490422C018FBF7A6F94A
:10E80000002867D1A869AE62001DA861A968686880
:10E81000FDF792F8A04202D1E968884209D00422AB
:10E8200012216B690C9800F07FF8FCF7F1FC0FB037
:10E83000F0BD384C6F460FCC0FC70FCC0FC7A26886
:10E84000616820680A920890334F0098203C099133
:10E85000B84206D128212046FDF76EF80A99884271
:10E860000AD000960196029603960496059606969F
:10E870000796089609960A960097284A6968914271
:10E8800001D1012000E0022001909142684601D1AF
:10E89000083000E018300160A9684160E9688160D3
:10E8A0002969C16028216846FDF746F80A9020468C
:10E8B000FBF71EF900280DD12C2269462046FBF7F4
:10E8C00045F9002806D12C2221466846F9F709FDB2
:10E8D000002809D0052212216B690C9800F024F859
:10E8E000FCF796FC0FB0F0BD00221221AB680C982B
:10E8F00000F01AF8C82001F0ADF8BFF34F8F0949B6
:10E900000748C860BFF34F8FFEE700005447002060
:10E91000784700200040000111C011CA00800001AA
:10E920000400FA0500ED00E010B582B06C462170DD
:10E930006270A370190AE170190C2171190E6171CE
:10E94000014606236A461F20FCF796F902B010BD67
:10E95000102819D230B40D4C83001B199D6989030E
:10E960002D0B2D03090D0D439D619969084D9209E9
:10E9700092052940920A11439961012261698240FE
:10E980001143616130BC70477047000000200240B5
:10E99000FF0FC0FFF3B5054681B00026408800F0A8
:10E9A00003F901000AD01C4F6A8800201423434356
:10E9B000DB195B8A934203D142262AE0402628E0F5
:10E9C000401CC0B20A28F1D3002E22D1002414200A
:10E9D0006043C019408AFF2806D0641CE4B20A2CA8
:10E9E000F5D30A2C14D014E02846083000901420E7
:10E9F0006043C0190E686B78AA880746A91DB04706
:10EA00000600EED1688878820298398A0180E8E7AA
:10EA10004B26304603B0F0BD3C4B0020028850042A
:10EA2000400CD20B01D009020843704710B40024F7
:10EA3000094A214614234B439B185B8A834204D125
:10EA4000142041438818C46803E0491CC9B20A294C
:10EA5000F0D3204610BC70473C4B002030B4FF235D
:10EA6000040AC5B20A490020142242435218128AED
:10EA7000AA4204D1142250434018438A03E0401CA8
:10EA8000C0B20A28F0D3200230BC184370470000FF
:10EA90003C4B0020084A11780A290AD2C900436871
:10EAA000891800688B6048601078401C1070012045
:10EAB0007047002070470000044C002030B4FF2352
:10EAC000040AC5B20A490020142242435218528A4D
:10EAD000AA4204D1142250434018038A03E0401C88
:10EAE000C0B20A28F0D3200230BC1843704700009F
:10EAF0003C4B0020F1B582B00299294E002000293C
:10EB000000D1307000250298002804D0012834D0AC
:10EB100002283ED10FE0294614225143214A2846BB
:10EB200009308C182082C0B209F434D1207C2146EF
:10EB300009F416D12DE02846142148431949002331
:10EB40004718B87C009030781C4600280DD9E000AA
:10EB50008019828800998A4202D1806880470346E2
:10EB6000641C3078E4B2A042F1D8002B02D059687E
:10EB700038468847387C09F431D11422094B6A435E
:10EB80000021D018FF24C160448299504160018166
:10EB900041816D1CEDB20A2DB5D303B0F0BD00006C
:10EBA000044C00203C4B002070B50146094DCEB20C
:10EBB00000202978044600290BD9E10049198A88E8
:10EBC000B24201D188688047641C2978E4B2A1422E
:10EBD000F3D870BD044C002070B5054600780028BD
:10EBE00013D00A4E2846F9F75DFB84B20D2C00D9EC
:10EBF0000D2471782346481C70702A460220FCF7C9
:10EC00003BF82D1928780028ECD170BD4C47002026
:10EC1000F8B5134E0F46756904463068001D00F0C4
:10EC200037FE601C07D1002F05D031680D48091D43
:10EC300000F0BBFEF8BD30682C1944603168AC426E
:10EC400004D2B068091D00F097FEF8BD7068091D78
:10EC500000F092FE306B8442F7D23463F8BD0000BE
:10EC600084470020EC580020F8B5856B1646044612
:10EC70000027026C002A11D0002E19D0E068F9F7A5
:10EC8000EDFA216CE068401AE0602268904202D2FE
:10EC90006068401AE060022E17D019E02068002852
:10ECA00016D1606801F088FC0746002060600FE024
:10ECB000A068F9F7D3FA216CA0684018A0606168D9
:10ECC000884205D32068A06002E0002D00D06D1EB0
:10ECD0006D1CA5633846F8BD114D124E124FE86801
:10ECE000002817D000F06EFEF068C468201D00F008
:10ECF000CFFD2869401E2861E868401EE86000F0EA
:10ED00006DFE206B00F078FE204600F075FEE8688E
:10ED10000028E7D138680128E1D900F08FFEDEE74E
:10ED200084470020D85800201058002030B41249E1
:10ED300000E011460A688242FBD34B685C188442AB
:10ED400003D1406818184860084643681C1894426C
:10ED50000CD10A4C2468A24206D052689A1842602C
:10ED60000A681268026002E0046000E0026081420A
:10ED700000D0086030BC7047D0470020C04700205A
:10ED8000F7B582B0039800260068002859D0039890
:10ED9000416802464968083241600092914201D1BF
:10EDA000496841604068C0680190039841684968BB
:10EDB0004160009A914201D149684160CF682420A6
:10EDC00002997043441804983D46002F01D11E4912
:10EDD0000D682560294634316160E96A2161296B3B
:10EDE000E161696CA1600023E96CA36161610528A0
:10EDF00013D015490A68954201D1237311E020739D
:10EE000003280ED1886B401C8863A86A002801D0B3
:10EE10000220207301F072FC03E02846FDF744F85D
:10EE20002073286B00210278A52A04D14278401C67
:10EE3000491CA52AFAD0880820840198761C8742AC
:10EE4000B3D1304605B0F0BD8447002003480068C8
:10EE5000401C72B600D0FEE7FEE70000D847002055
:10EE6000F8B5054600F0AEFD2E4640360524345771
:10EE7000002C0FDD2F462437686A00280AD0384658
:10EE800001F00AFC002801D000F06CFE641E64B2A0
:10EE9000002CF1DC0027FF43777100F09FFD00F0AC
:10EEA00091FD04243457002C10DD284610300090CA
:10EEB000286900280AD0009801F0EEFB002801D054
:10EEC00000F050FE641E64B2002CF1DC377100F0DB
:10EED00085FDF8BDF8B50446002500F0BDFE374EAF
:10EEE00000273068364A002801D0F0681BE0052171
:10EEF00034480903430705D0C01DC008314BC0008A
:10EF0000C31AC91A41180839C908C90057601060E6
:10EF100031604F600B1A0F6043600160B3600120E5
:10EF2000C0077360F06004423FD1002C3DD0204602
:10EF30000830410708D04107490F0823591A08181B
:10EF4000410701D072B6FEE700282ED071688842D2
:10EF50002BD81B49146801E021461446626882429E
:10EF600002D22268002AF7D1326894421DD00D687F
:10EF700022680A60616808350A1A102A09D921181E
:10EF80004B0701D072B6FEE74A6060600846FFF7A3
:10EF9000CDFE61687068401A7060B268904200D21D
:10EFA000B060F06827600143616001F0A7FB68076B
:10EFB00001D072B6FEE72846F8BD0000C047002029
:10EFC000D04700200059002004490868002803D0D9
:10EFD0000868026D521C026508687047844700206B
:10EFE00010B40124031F24061C601B1F1960191F85
:10EFF000034B0B6014390A6010BC403870470000A6
:10F000004DEE000170B5064614460D464720FFF749
:10F010000DFD0369002B0DD01879B04207D1587946
:10F020002880981D2060002B04D0002070BD1B6834
:10F03000002BF1D10020288020600A2070BD000044
:10F0400070B516460C46104608F434D6002813D185
:10F050004720FFF7EBFC05460623324619460748D2
:10F0600008F46AD5A988628889180180A18841803E
:10F07000A179017108F49CD5002070BD180C000026
:10F08000F7B506460D464720FFF7D0FC0469074652
:10F09000002C14D02079B0420BD16079A8420CD05A
:10F0A000384621461030F9F745FD204608F434D49F
:10F0B00005E02468002CEDD101E0002C0AD128469F
:10F0C0000121083008F4B2D4044601463846103015
:10F0D000F9F736FD267165712A46A01D0299F9F7E8
:10F0E000BDF8002003B0F0BDF8B5C5680124287F45
:10F0F0000F4601281ADD0E4E2046162250430246C6
:10F10000296A10328A5A5204920F0BD10A5C401CB1
:10F11000085C00021018B04204D1E1B20022384667
:10F1200000F03EF9287F641CA042E5DCF8BD000039
:10F1300002290000F8B5C5680124287F0F46012880
:10F140001ADD0E4E2046162250430246296A10321E
:10F150008A5A5204920F0BD10A5C401C085C0002D0
:10F160001018B04204D1E1B20022384600F018F97C
:10F17000287F641CA042E5DCF8BD000002290000E5
:10F1800070B5C46805462069002803D00020002817
:10F1900002D00EE00120FAE7264610363046F9F795
:10F1A000B7FC08F4B9D32069002808D00021002951
:10F1B000F4D00020E860204608F4AED370BD0121F1
:10F1C000F5E710B504464720FFF730FC82790021AF
:10F1D000A24202D98088001981B2084610BD70B5DC
:10F1E00004460D464720FFF721FC01468088802217
:10F1F000A04206D889794118A14202D9201A287064
:10F200000022104670BDFFB585B00E9D06462978D8
:10F2100001208840401E049018460E210840328A82
:10F2200069681F46403001920023039000930291C9
:10F230002B7804AAA9680698F9F7A0FC009000288A
:10F240002AD10121282008F4F1D30446AA6869686C
:10F25000286862622162E061F46006980188A180FA
:10F26000217FA171F80701D00120C003079908434D
:10F270002080308A608047207082304600F0AAF8F3
:10F2800020461030F9F750FC217F206A00F008F882
:10F29000308A002108F420D5009809B0F0BD0000A4
:10F2A000F3B583B00020019004980125012845DDC5
:10F2B0001621039A69438818028A5204920F39D1A1
:10F2C000039A4078515C000209181D48814231D1EF
:10F2D00001A80290EFB204264720FFF7A7FB009099
:10F2E0000469002C14D02079B8420BD16079B04267
:10F2F0000CD0009821461030F9F71CFC204608F489
:10F300000BD305E02468002CEDD101E0002C0AD1DC
:10F3100030460121083008F489D30446014600989C
:10F320001030F9F70DFC277166713246A01D029965
:10F33000F8F794FF04986D1C8542B9DB05B0F0BD69
:10F340000229000000487047AC0D010170B5064667
:10F3500010480D46007800281AD04720FFF7AEFB72
:10F36000A91D8BB2014603220B4808F4E5D30446DD
:10F370000A482A468078207001206070052060804D
:10F38000A5803146A01DF8F769FF204608F410D487
:10F3900070BD00003747002006470000844D002064
:10F3A00070B584B00E461446054601AA694630463B
:10F3B000FFF728FE6846028802A80199F8F74EFF79
:10F3C00002A844550246684601883046FFF758FEB9
:10F3D00004B070BD10B504464720FFF727FB044971
:10F3E000216009216181183060600120208110BDF9
:10F3F000BC0D0101FFB583B00C464720FFF716FB9B
:10F400000546808861882678401887B2059808F4F8
:10F4100051D4012807D03846FDF758FE6946FFF75A
:10F42000DEFE002802D0022007B0F0BD01210598C1
:10F4300008F452D40C3C0020AC6028736846007875
:10F44000687301AA02A9FFF7DDFDA86801990446C7
:10F45000895D0C34890720D5A188C28808318BB218
:10F460003102C1200001891D08F466D3064613202D
:10F470003070A88861884018B080A088F08030463D
:10F48000A288A11D0830F8F7E9FE304608F490D3B1
:10F490000121059808F420D401E008F43DD20120B0
:10F4A00007B0F0BD10B5FCF7C3F8002010BDFFB5E4
:10F4B00083B00C464720FFF7B9FA0546808861887B
:10F4C0002678401887B2059808F4F4D3012807D0AD
:10F4D0003846FDF7FBFD6946FFF781FE002802D0A4
:10F4E000022007B0F0BD0C3CAC602E73684600787B
:10F4F000687301AA02A9FFF785FDA868019904466F
:10F50000895D0C34890720D0A188C28808318BB26C
:10F510003102C1200001891D08F40ED306461220D5
:10F520003070A88861884018B080A088F08030468C
:10F53000A288A11D0830F8F791FE304608F438D3B0
:10F540000121059808F4C8D301E008F4E5D10120B1
:10F5500007B0F0BD10B50C464720FFF767FA80886A
:10F560006188A31D401880B2A1880022FBF7F8FF34
:10F57000002010BD10B508460022898801E0521C09
:10F5800092B29142FBD84288022A0DD0062A0ED1AF
:10F5900002290CD18179C07908180649012801D0C7
:10F5A000002804D1087002E0801DFBF7A5FA0020B6
:10F5B00010BD000037470020F8B518460D4601463B
:10F5C00005260BA70D230C4808F4B6D204460020EC
:10F5D000A07128782070A6806888608032463946FD
:10F5E000E01DF8F73BFE204608F4E2D20020F8BD0B
:10F5F0004E53494E470000000547000070B51646BF
:10F600000C46104608F456D3012818D1A1791A489F
:10F61000002916D02178062309023246891D08F4F4
:10F620008BD20546A078FFF7CCFD2880802028717A
:10F63000284608F4BDD20021304608F44DD30020FE
:10F6400070BDA1883246891D8BB221780902891DBF
:10F6500008F472D20546A078FFF7B3FD2880002099
:10F660002871A0886880A288E11D681DF8F7F6FD62
:10F67000284608F49DD2DEE7140C000010B50124E2
:10F6800000206407206008F4ADD12E4802882E487F
:10F690000168002008F432D22C4802882C48016806
:10F6A000012008F42BD22B48008882B22A48016836
:10F6B000022008F423D22948008882B22848016831
:10F6C000032008F41BD22748416AF022114341620B
:10F6D00025481BF405D2264824490160254941618B
:10F6E000254981602549C160254981612549C1615C
:10F6F000264925488863FDF7D7FD2068C0B2F9F791
:10F7000043FA23480078002806D000201BF42ED5A9
:10F7100001460020F9F73EFA2068C0B2F9F740FA36
:10F72000F9F744FA2068C0B21BF4ACD22068C0B22A
:10F730001BF4B6D22068C0B21BF474D40120206040
:10F7400010BD00001C010020180100202401002031
:10F750002001002034010020300100202C01002075
:10F760002801002040250240740200205002500071
:10F770008080024000080F0058086A00420500001F
:10F780000F0505060F000F034000D0004080024027
:10F7900062000020F0B5314C83B0E06980075AD593
:10F7A00002202062A56B08201BF484D501201BF4E5
:10F7B0008FD52B490027086940194608B219801ACD
:10F7C000086128480068F8F7E1FF0022264BF8F7A7
:10F7D0005DFF019100903E212846F9F7EDF980196F
:10F7E0007941F8F7E1FF019B009AF8F7E7FEF9F796
:10F7F00003F805461D4A0023F8F7EEFC06461B49B0
:10F80000F9F7DAF91A49281A081A81B222041948B4
:10F81000324342600160206B082188430843206323
:10F82000A069072109078843A061A16901208143DC
:10F830000143A1612062FDF737FD0F48104A0078AF
:10F84000410041180D4808184178D1610D49807870
:10F85000C8600D48077003B0F0BD00000080024092
:10F86000A80200209000002000408F40710200009C
:10F87000700200004080024010400020CC0C0101CA
:10F8800040250240802502408000002070477047DC
:10F890004368826801699A60836842685A604A686E
:10F8A000824201D182684A60002202610868401EDB
:10F8B0000860086870470000014800697047000050
:10F8C00084470020F8B51746204A06460024906B6E
:10F8D0000725401C90631069814232D314206D1EAD
:10F8E0001B49684341182420604380190122FFF717
:10F8F00047FA0419002DF1D12420144D60438019DA
:10F9000002226968FFF73CFA041924206043801939
:10F910000222A968FFF734FA0419242060438019F1
:10F9200004220C49FFF72CFA0419242060438019A3
:10F9300003220949FFF724FA0419002F01D00020FF
:10F94000386000F0DBFE2046F8BD00008447002050
:10F9500010580020D8580020EC58002001460831EB
:10F9600000224160D243C1608260016100210160D8
:10F97000704700210161704730B40C68621C02D0EE
:10F980000246083202E0026904E01A4653681D6824
:10F99000A542FAD953684B6099608A60516008614A
:10F9A0000168491C016030BC704742684A60936836
:10F9B0008B6093685960916008610168491C01601F
:10F9C0007047000072B604480168491C0160BFF32B
:10F9D0004F8FBFF36F8F7047D847002005490868E5
:10F9E000002804D0401E086000D162B6704772B68D
:10F9F000FEE70000D847002000281CD070B5044660
:10FA00000D4D083C6068E968084201D172B6FEE716
:10FA10002268002A01D072B6FEE78843606000F0D9
:10FA20001BF960686968401868602046FFF77EF936
:10FA300000F064FE70BD7047C047002001200449FB
:10FA400000074860BFF34F8FBFF36F8F7047000010
:10FA500000ED00E010B500280FD009498A6B002A9C
:10FA600001D072B6FEE78A6B521C8A630021FFF751
:10FA7000CFF800F043FE002801D1FFF7DFFF10BDF3
:10FA80008447002002498A6A0260496941607047E0
:10FA900084470020F0B585B00027054607702C4844
:10FAA00001690291006924214843FFF713FA060017
:10FAB0004CD000220299FFF705FF0397029000281F
:10FAC00041D90398242148438019017B052911D28B
:10FAD0000A007A44127992189744020406080A0030
:10FAE000582408E0522406E0422404E0532402E0B3
:10FAF000442400E0002441682846F8F7FFFB28462C
:10FB0000F8F7D0FB0F2804D220212954401C0F28DD
:10FB1000FBD32F542D180398242148438019018CBE
:10FB2000826801920091036922460AA12846FAF7E9
:10FB300053FA2846F8F7B6FB451903980299401C7A
:10FB400003908842BDD33046FFF756FF05B0F0BDA5
:10FB50008447002009256309257509257509257540
:10FB60000D0A0000014901204862704784470020C7
:10FB700010B50C46002809D0054909681831FFF76F
:10FB8000FBFE01212046FFF743F810BD72B6FEE7E9
:10FB90008447002070B50B4604002FD0226D002A48
:10FBA0000ED0E16C994200D21946E06A884225D015
:10FBB000012A23D1124D2A68944203D172B6FEE77E
:10FBC00072B6FEE7E162A269002A02DB0722511A3F
:10FBD000A16114220B4E50436169801981420DD1FD
:10FBE000201DFFF755FEE06AA969884200D9A86187
:10FBF000142148438019211DFFF7D7FE70BD000076
:10FC0000844700201058002010B582B00D48002411
:10FC10000190234680220CA100940D4800F090FB37
:10FC2000012803D0401C0BD172B6FEE772B600214A
:10FC30000848C94301630121C161446100F052F8E1
:10FC400002B010BDB847002049444C4500000000F8
:10FC5000D9EC0001844700200248816B491C816374
:10FC60007047000084470020164B986B002802D094
:10FC7000012058627047002058629869142102469A
:10FC80004A4311498A58002A0AD1002806D0142272
:10FC9000401E42438A58002AF7D001E072B6FEE7C0
:10FCA000142210B4424351184A680C465268083472
:10FCB0004A60A24201D152684A60D16819609861D5
:10FCC00010BC70478447002010580020014840684D
:10FCD00070470000C047002001488068704700005E
:10FCE000C047002070B50F48016AFF22120411437B
:10FCF0000162016A1202114301620B4C0025256169
:10FD0000A5610A487D21C9000068F8F73BFA401E4A
:10FD100060610720206106480560F8F7E9F90020D6
:10FD200070BD000000ED00E000E000E000400020B9
:10FD3000D847002010B502460021012000F00CF841
:10FD4000041E07D00021416001600B460A46C160D5
:10FD500000F05BF8204610BDF8B517460E460500CA
:10FD600016D0002E16D070435030FFF7B3F80400C1
:10FD70000CD020465030002E0ED020602664204645
:10FD80000121E56300F00AF84C2007552046F8BD34
:10FD900072B6FEE70020E7E72460EFE770B50D4696
:10FDA000040026D0FFF70EFE216CE06B484321686B
:10FDB000411861600021A1632168A160E06B216CA2
:10FDC000401E48432168224641180020C04340326B
:10FDD000E1601071507120461030002D0BD0FFF7FC
:10FDE000BDFD20462430FFF7B9FDFFF7F7FD0120E8
:10FDF00070BD72B6FEE721690029F6D000F04CFC18
:10FE00000028F2D0FFF71AFEEFE7FFB5002783B016
:10FE10000446002803D00498002802D006E072B6F9
:10FE2000FEE7206C002801D072B6FEE70698022893
:10FE300004D1E06B012801D072B6FEE700F03CFB74
:10FE4000002804D10598002801D072B6FEE72046AC
:10FE50002546103040350290FFF7B4FDA06BE16BF2
:10FE6000884208D30698022805D0059800284AD071
:10FE7000002F4BD04EE0069E0499A56B0027226C04
:10FE8000002A11D0002E19D0E068F8F7E7F9E168F0
:10FE9000206C091AE1602268914202D26168081A56
:10FEA000E060022E17D019E02068002816D16068A3
:10FEB00000F082FB0746002060600FE0A068F8F7C2
:10FEC000CDF9216CA0684018A0606168884205D314
:10FED0002068A06002E0002D00D06D1E6D1CA5639F
:10FEE000606A002806D02046243000F0D5FB0028A8
:10FEF00002D103E0002F01D0FFF7A0FDFFF76EFD58
:10FF0000012007B0F0BDFFF769FD20E06846FFF76C
:10FF1000B9FD0127FFF762FDFFF79EFEFFF752FDD7
:10FF200004202856401C00D1287105202856401C6A
:10FF300000D16871FFF752FD05A9684600F0CEF9BF
:10FF4000002807D02046FEF78BFF00F0D7FB0020EB
:10FF500007B0F0BDFFF736FDA06BE16B884201D121
:10FF6000012600E00026FFF739FD002E0ED005998E
:10FF70000298FFF7FDFD2046FEF772FF00F0BEFB82
:10FF8000002800D068E7FFF759FD65E72046FEF737
:10FF900067FF00F0B3FB5FE7FFB583B01E4617466F
:10FFA000040003D00498002802D006E072B6FEE7F1
:10FFB000206C002801D072B6FEE7022E04D1E06B5F
:10FFC000012801D072B6FEE7F8F7A6F80190A06B01
:10FFD000E16B884208D3022E06D000240198F8F77E
:10FFE0009FF8204607B0F0BD204640300525009020
:10FFF0004557324620460499FEF736FE681C04D069
:020000040101F8
:1000000000986D1C45710124E8E7606A0028FAD069
:100010002046243000F040FB0028F4D0002FF2D01E
:1000200001203860EFE7F7B5002784B004460028C8
:1000300003D00598002802D006E072B6FEE7206CD7
:10004000002801D072B6FEE700F036FA002804D18D
:100050000698002801D072B6FEE7204625462430D7
:1000600040350290FFF7AEFCA66B002E21D0226C2B
:10007000059B002A0BD0E0688018E0606168884228
:1000800001D32068E06001461846F8F7E7F8761ECD
:10009000A6632069002807D02046103000F0FCFA43
:1000A000002801D0FFF7CAFCFFF798FC012007B039
:1000B000F0BD0698002802D0002F05D008E0FFF719
:1000C0008DFC002007B0F0BD6846FFF7DBFC012780
:1000D000FFF784FCFFF7C0FDFFF774FC04202856EF
:1000E000401C00D1287105202856401C00D16871A1
:1000F000FFF774FC06A9684600F0F0F8002811D05C
:100100002046FEF7ADFE00F0F9FAFFF75BFCA06BAE
:10011000002827D00026FFF761FC002EA2D0002087
:1001200007B0F0BDFFF74EFCA06B002812D00026F0
:10013000FFF754FC002E0FD006990298FFF718FD28
:100140002046FEF78DFE00F0D9FA00288AD1FFF78D
:1001500075FC87E70126EBE72046FEF781FE00F0FD
:10016000CDFA7FE70126D6E7F3B5002785B0044630
:100170000097002804D0206C002803D072B6FEE758
:1001800072B6FEE700F098F9002804D1069800281E
:1001900001D072B6FEE72046254624304035019056
:1001A000FFF710FCA06B002817D0401EA06320684A
:1001B000002802D1FEF708FF60602069002807D000
:1001C0002046103000F068FA002801D0FFF736FC16
:1001D000FFF704FC012007B0F0BD0698002802D00C
:1001E000002F0AD00DE00098002801D072B6FEE77B
:1001F000FFF7F4FB002007B0F0BD02A8FFF742FCB8
:100200000127FFF7EBFBFFF727FDFFF7DBFB0420E0
:100210002856401C00D1287105202856401C00D1CA
:100220006871FFF7DBFB06A902A800F057F8002869
:100230001BD02046FEF714FE00F060FAFFF7C2FB69
:10024000A06B00283ED00026FFF7C8FB002EA7D0E9
:10025000009800283ED0FFF7B5FB606A002833D035
:10026000206B07210068091A2FE0FFF7ABFBA06B9A
:10027000002808D00026FFF7B1FB002E1CD0206814
:10028000002802D009E00126F5E7FFF79BFB606834
:1002900000F0C6F90090FFF7A1FB06990198FFF75F
:1002A00067FC2046FEF7DCFD00F028FA002800D0AD
:1002B00076E7FFF7C3FB73E72046FEF7D1FD00F0BA
:1002C0001DFA6DE70126BFE700216068FFF762FCB9
:1002D000FFF784FB002007B0F0BD0000F8B50D4625
:1002E000040012D0002D12D0FFF76CFB134E726980
:1002F00063682868D11A471C0BD02768B66AB742D2
:1003000009D0934207D8012413E072B6FEE772B613
:10031000FEE700240DE0884208D9401A286007480B
:10032000816A216040696060002402E000200124AD
:100330002860FFF753FB2046F8BD000084470020EB
:10034000FFB585B090000F9F0E9D0290FEF7C2FD95
:1003500006001ED05C20FEF7BDFD040016D026630B
:10036000059901910899009130460299069EA522AF
:100370000391F7F785FF0399206B091F4018C00808
:10038000C0000290400708D072B6FEE73046FFF783
:1003900033FB0020C04309B0F0BD2118325C20318E
:1003A0000A75315C002902D0401C1028F5D326467E
:1003B00000204036F070072D00D30625E5620020AE
:1003C000E5642065201DFFF7D4FA20461830FFF7BA
:1003D000D0FA24610720411B6462A161002161659C
:1003E0003176009A01990298FEF7FAFD2060002FFD
:1003F00000D03C602546FFF7E5FA284E3069401CE6
:1004000030613068264F002803D0F069002821D0E1
:1004100026E035603069012822D100241420604391
:10042000C019FFF79BFA641C072CF7D31D48FFF790
:1004300095FA1D48FFF792FA1C48FFF78FFA1C48FF
:10044000FFF78CFA1B48FFF789FA164870601430E2
:10045000B06005E03068E96AC06A884200D835605B
:10046000F06A401CF0626864E86AB169884200D9A9
:10047000B06114214843C019291DFFF796FAFFF710
:10048000ADFAF069002806D03068E96AC06A88428F
:1004900001D2FFF7D3FA012009B0F0BD8447002054
:1004A000105800209C580020B0580020C45800204C
:1004B000D8580020EC5800200648C169002904D013
:1004C000806B002803D00020704701207047022075
:1004D00070470000844700200148406970470000D1
:1004E00084470020F8B5324F0026B86B002808D0AA
:1004F000386A401C3862786A002800D001263046ED
:10050000F8BD7D696D1C7D6115D178680068002893
:1005100001D072B6FEE77868B9687960B860B86AE9
:10052000401CB86278680068002813D07868C068FA
:10053000C06840683863386B854211D378680068BA
:1005400000280AD07868C068C4686068854211D203
:10055000386305E00020C043ECE70020C043386367
:1005600038681421C06A4843124908580128C2D982
:100570000126C0E7201DFFF78BF9A06A002803D0F1
:1005800020461830FFF784F9E06AB969884200D93B
:10059000B8611421484307494018211DFFF705FAA7
:1005A000E06A3968C96A8842C8D30126C6E70000F4
:1005B000844700201058002070B500210446002810
:1005C00028D0154D2868844201D072B6FEE7206D10
:1005D000002808D0401E2065E36CE26A9A4219D0D8
:1005E000002802D016E072B6FEE7201DFFF750F992
:1005F000E06C0721E062081AA061E06AA9698842FC
:1006000000D9A8611421484304494018211DFFF76F
:10061000CCF90121084670BD844700201058002005
:1006200070B504460020002C2AD0194DE16A2A68D2
:10063000D26A914225D2A069002804DB28680721EC
:10064000C06A081AA061E06A1422124E5043616920
:100650008019814210D1201DFFF71AF92868C06A5D
:10066000E062A969884200D9A86114214843801931
:10067000211DFFF79AF902E02868C06AE0620120B4
:1006800070BDE16C2A68D26A9142F8D370BD000057
:10069000844700201058002070B5C068C468002C42
:1006A0000BD0204618300646FFF7F2F8104DA86B25
:1006B000002804D031460F480EE072B6FEE7201D38
:1006C000FFF7E6F8E06AA969884200D9A861142119
:1006D000484309494018211DFFF767F9E06A296876
:1006E000C96A884202D90120686270BD002070BDCD
:1006F00084470020C458002010580020F8B52E4D23
:100700000027A86B002808D0FFF75CF9A86B401EF3
:10071000A863A86B002802D046E072B6FEE72869FD
:10072000002841D0254E306800282AD0F068C468DF
:1007300020461830FFF7ACF8201DFFF7A9F8E06A53
:10074000A969884200D9A861142148431C4940186E
:10075000211DFFF72AF9E06A2968C96A884201D396
:100760000120686230680028E0D1002C09D0686858
:100770002946006800281BD04868C068C0684068E7
:1007800008632C6A002C09D00126FFF7ABFE002875
:1007900000D06E62641EF8D100202862686A0028CA
:1007A00002D00127FFF74AF9FFF718F93846F8BDDC
:1007B0000020C043E4E7000084470020C458002024
:1007C0001058002040BA7047C0BA70470138FDD1B8
:1007D00070470000F7B50325AD06286A82B01646BB
:1007E0000C46400840002862286A0221084328621B
:1007F000286A8007FCD46620686001272F61A86AF8
:10080000C005FCD5992068602F61A86AC005FCD599
:10081000FF209130FFF7DAFFFF230133AB62684618
:10082000EF60352169602F61A96AC905FCD5AB620B
:10083000A969EF60C9B205226A602F61AA6AD20570
:10084000FCD5AB62AA690902D2B211430180C80784
:1008500002D0032005B0F0BDAB626869FF2108310A
:10086000884368616869C91E08436861029800028C
:10087000483068600820A860EE602F61A86AC00553
:10088000FCD5FF200130A8620023F61CB0080ED072
:10089000B2081148006899006054060A09194E70A0
:1008A000060C000E8E705B1CC8709A42F1D8FF20B7
:1008B0000130A8626869FF2108318843686168696E
:1008C00038436861286A800880002862286A3843B3
:1008D0002862002005B0F0BD8000000C03208006D7
:1008E0004169FF22083291434161426901210A4373
:1008F0004261026A920892000262026A0A4302623C
:1009000070470000002003218906096A4908490050
:100910000322920611621146096A02221143032240
:100920009206116200BF03218906096A0222114062
:100930000229F8D0D1010322920691620321D160ED
:100940009F2151600121116100BF03218906896A3D
:10095000FF22013211409142F7D1032292069162A7
:10096000114688694969FF220832914303229206A1
:1009700051611146496901221143032292065161D6
:100980001146096A8908890011621146096A012223
:100990001143032292061162704700000000010219
:1009A00000000000010203040138FDD1704700007F
:1009B000F0B40324A406236A5B085B002362236A65
:1009C00002252B432362236A9B07FCD4FF230133B8
:1009D000A3626569DE1DB543656165691E1D35430A
:1009E000656100026B3060600820A060E260012653
:1009F0002661A06AC005FCD5A3620023D21C900822
:100A00000ED095080F4800689A008854070A5218BB
:100A10005770070C000E97705B1CD0709D42F1D888
:100A20006069FF210831884360616069304360611B
:100A3000206A800880002062206A30432062F0BC77
:100A4000002070478000000CF8B506460120002504
:100A5000C004864201D90520F8BD0324A406206AFB
:100A6000400840002062206A022108432062206A78
:100A70008007FCD4FF270137A76200F0BBF80028ED
:100A800001D0032515E00620606001212161A06AE4
:100A9000C005FCD5A7623002203060602161A06AE9
:100AA000C005FCD5A7620C4800F0C8F8002800D1AA
:100AB00002256069FF210831884360616069012176
:100AC00008436061206A800880002062206A084331
:100AD00020622846F8BD0000E6960100F7B50646FC
:100AE0000120C00482B01546864202D9052005B017
:100AF000F0BD03208006016A490849000162016ACD
:100B0000022211430162016A8907FCD4FF210131ED
:100B10008162F2B28C1AA54200D8ACB20398009060
:100B200000F068F8002840D1062148064160012104
:100B30000161816AC905FCD5FF21013103208006CE
:100B400081624169FF220832914341614169042277
:100B500011434161310232314160C4600022002CF6
:100B600016D9009887183B78F87819467B780006E4
:100B70001B021943BB781B04194301430802F9788F
:100B8000000A0906084319490860121DA242E8D369
:100B90000121032080060161816AC905FCD5FF217E
:100BA00001318162124800F049F8A54209D003984A
:100BB000361900192D1BFF2401340390A542ADD82E
:100BC000ABE7032080064169FF220832914341616F
:100BD0004169012211434161016A8908890001626A
:100BE000016A11430162002005B0F0BD8000000CD5
:100BF0001A06000038B40125032080066A46C56045
:100C0000352141600561816AC905FCD5FF240134A5
:100C100084628169C560CBB2052141600561816A4A
:100C2000C905FCD5846280691902C0B2014388B24B
:100C30001180C00700D0012038BC7047F8B40021F3
:100C40000125032292066B46D56035245460156158
:100C5000946AE405FCD5FF27013797629469D56053
:100C6000E4B2052656601561966AF605FCD59762D2
:100C700096692402F6B234431C80E30722D08142F5
:100C800002D9F8BC00207047032292066B46D5605B
:100C9000352454601561491C946AE405FCD59762BB
:100CA0009469D560E4B2052656601561966AF6052A
:100CB000FCD5976292692402D2B21443A2B21C807E
:100CC000D207DCD1F8BC01207047000000171300E8
:100CD000171000170E00170900170400170000175F
:100CE0001801171401171501171900000028000238
:100CF000000000000328000200000000292A000272
:100D0000008080000328000200000000242A000266
:100D1000008080000328000200000000252A000255
:100D2000008080000328000200000000272A000243
:100D3000008080000328000200000000262A000234
:100D4000008080000328000200000000282A000222
:100D5000008080000328000200000000232A000217
:100D60000080080003280002000000002A2A000278
:100D7000008008000328000200000000502A000242
:100D800000800700CDBB00015BBB000159BB000127
:100D900057BB00010014000075BC0001130C0000DB
:100DA00019CE00010314000031BD000107F200015B
:100DB00081F1000135F10001E9F00001130C0000A0
:100DC000DDCE0001150C0000BDCF0001170C0000A6
:100DD000F5CC0001000C000035CD000106470000F5
:100DE000AFF400010347000055F50001084700007B
:100DF000F5F300010E47000041F000010547000037
:100E0000FDF50001FFFF0000ADB30001130E00006F
:100E100035C00001150E000045BF0001170E00008F
:100E2000B5C40001190E00008DC40001040E0101BB
:100E300005000000F7B586B0002002905C4815461A
:100E400004695C480E46824201D9054602E0002D45
:100E500000D10125002C08D0A1880698814204D138
:100E6000E088B04201D101200290534803908446AB
:100E70000698010431430020002C1CD00A0CA788DE
:100E80008BB2974207D1E7889F4204D1002807D050
:100E90002168016007E020462468002CEFD10AE0B9
:100EA000614622680A602168002902D00020206083
:100EB00001E061464860002C07D10221102000F0BB
:100EC00095F8069981800446C6802801052100F026
:100ED00077F807467D200E464643EFF31085012044
:100EE00080F31088684600F087F885F31088009832
:100EF0000490C0190501019927202D098E190001C0
:100F00000591864203D96D1C2D012D09361AE66024
:100F1000A5600398294F86460020844670460068E5
:100F2000002813D0A268E1680091C368816801932A
:100F3000531A1B011B09BB420AD2914203D1019AE9
:100F40000099914204D984460068E9E772465460EA
:100F500020606046002801D0046001E071460C600A
:100F6000134802990069002901D1A04203D1C16848
:100F7000806800F047F8EFF31084012080F31088B8
:100F800002A800F039F884F31088039902980191BF
:100F9000291A090109090090B94204D2A84205D1D1
:100FA0000198864202D8032000F032F809B0F0BD63
:100FB000C8010020FFFF7F02D8010020FFFFFF07CC
:100FC00030B50B46014600202022012409E00D46E1
:100FD000D5409D4205D31D469540491B2546954069
:100FE00040191546521E002DF1DC30BD03B40148F6
:100FF000019001BD2D7A010003B40148019001BDAB
:101000005DB6020003B40148019001BD9DB6020027
:1010100003B40148019001BDAD78010030B4C3684C
:1010200082688868084D141A2401C9682409AC42F2
:1010300003D2904204D18B4202D830BC01207047C9
:1010400030BC002070470000FFFFFF070A0C8388B8
:1010500089B2934204D1C088884201D101207047EF
:101060000020704770B4054600680022002810D0A8
:101070000B0C86888CB29E4207D1C688A64204D14A
:101080000168002A07D0116006E0024600680028C7
:10109000EFD170BC704729600168002903D000219E
:1010A000016070BC70476A6070BC7047F0B5104F4B
:1010B000026886460025002A10D0C8688C689368AC
:1010C0008446E01A00010009D668B84208D2A3425B
:1010D00001D1B44504D915461268ECE77046416069
:1010E0000A60002D01D02960F0BD70460160F0BD9E
:1010F000FFFFFF0770B584B004460E46EFF310857E
:10110000012080F3108802A8FFF776FF85F310888E
:1011100002980399024600900191A01A0001074924
:101120000009884204D2A24205D10198864202D821
:10113000012004B070BD002004B070BDFFFFFF07A8
:1011400030B583B00446EFF31085012080F310889A
:101150006846FFF751FF85F3108801990098616098
:10116000206003B030BD0000002800020000000035
:101170000328000200000000002A000A008020006E
:101180000328000200000000012A00020080020083
:101190000328000200000000042A0002008008006A
:1011A0000328000200000000A62A000200800100BF
:1011B0000328000200000000C92A0002008001008C
:1011C00000280002000000000328000200000000C8
:1011D000052A0020008004000229000A0000020005
:1011E0000328000200000000292B000A00801000E4
:1011F00003280002000000002A2B000200801000DB
:10120000FFFF000095AE0001A40D000059C70001CA
:10121000A50D00008DC700011A0D0000A5CC00012E
:10122000150D0000EDC70001000D000019C80001F8
:101230001C0D0000DBCC0001A70D0000F9CB000164
:10124000A80D0000E7CC0001020C0000CDCD00018C
:10125000000C0000A5CD0001010E0000D1C200016C
:101260000F0E00008DC60001110E0000F1C6000136
:101270002C0E000071C60001030E000029C40001FD
:101280000A0E0000E5C50001300E000065C6000131
:101290000C0E000019C70001000E00003DC2000145
:1012A000090E000065C20001010F000065B10001D8
:1012B000020F00005DAD0001030F000049B1000105
:1012C000040F00004DE30001001201013647002029
:1012D0000100190002140000ADBD0001D41201018B
:1012E00001000000981301010300000001102EC747
:1012F0008A0E7390E111C2086027000000280000E8
:1013000000000000000000000000000000020000DB
:1013100000000328000000000000000000000000A2
:101320000000000A0000000001002EC78A0E739022
:10133000E111C20860270000000400C0000201297A
:101340000000000000000000000000000000000A93
:1013500000801400032800000000000000000000CE
:1013600000000000000A0000000002002EC78A0EE4
:101370007390E111C20860270000001000C0000255
:101380000229000000000000000000000000000032
:10139000000A00801400000004470000B9F50001B5
:1013A0000A47000075F5000107470000A5F4000199
:1013B000D0140101D814010155930001B8140101A2
:1013C000A014010181950001C01401013014010134
:1013D00099940001C8140101F4130101099200015C
:1013E0009C1401016C140101C99300010102030462
:1013F0000506000073686F77206465766963652071
:10140000696E666F202874656D702F7664642F6630
:10141000616E2C2073616D6520617320424C452004
:10142000494E464F5F515545525920616C6C290019
:1014300073686F77204672656552544F53207275FA
:101440006E74696D6520696E666F202875707469A9
:101450006D652F7461736B732F686561702F746194
:10146000736B206C69737429000000006C65642044
:101470003C317C323E203C6F6E7C6F66667C746FC4
:1014800067676C653E3A20636F6E74726F6C2062A2
:101490006F617264204C4544000000006C6564007C
:1014A00073686F77206669726D7761726520766503
:1014B0007273696F6E00000076657273696F6E00FB
:1014C000737973696E666F00646576696E666F0026
:1014D00068656C70000000006C69737420616C6C4E
:1014E00020636F6D6D616E64730000000C15010167
:1014F00000400020E00700008C8A00010C1B010165
:10150000E047002020690000F02A0000A0060090BB
:10151000D00300011005A00000FF01D20001000669
:1015200051C20200200001302B11D80D4908684932
:101530006813F008FB0498EFF78EFF0446C188801B
:1015400088FF22FFF79DFD2046FFF73AFCB3E70531
:10155000B0F0BD98100707D8010020C8042029303A
:10156000D70200004B1847FBFD064605203070757A
:10157000800099B181301D3946E5F773FD3046F999
:10158000F70EFF0E22294642200445FD0740301188
:101590002E0CD0534B052203212846FDF733FE12B3
:1015A0001E40274B75002D05D0398F002902D00031
:1015B00099897900E000211176FAF74BF8044D285B
:1015C00059F9F7FBFE002028518010060004002086
:1015D0000777107838B5049C0094014CA04738BDBB
:1015E0005143F84A26468F1839462036FD6D707DE6
:1015F00080311191C97FA0370E912246397815327A
:101600000F92F14A109203292BD0002873D0F17D5C
:101610000F980CF00DF800286FD068886946088391
:10162000F0B597B008780C460F90002014900F98F2
:1016300048214843FE49224640180646803610900D
:10164000F17F0091C56DA0301690014E100A27461B
:1016500012922037F74A1552146C2AD061783C292F
:1016600049D0432947D0787D00287DD0F97D129854
:1016700000F0FCF9002878D0698868468184687A8F
:10168000297A000409020843E97908430690A97AF7
:1016900008A84172E97A8172297BC17229460D310D
:1016A0000E380E9100F02FFAA878400733D50021AC
:1016B00032E0907E012806D0507E401E0006000ECB
:1016C000507603D006143004DB480106141200F0F3
:1016D000D2F9169A01211170A978D448C9075C364D
:1016E00090264823594308180022A0300270FF209A
:1016F000F07752E001220270A878CC49C0074CD0A4
:101700000098482358434020101442E0E97C08A880
:101710000173297D4173697D8173A97DC108100D15
:101720000174297E4174697E8174B189BC10228163
:10173000F189C181318A0182109940318A8F828377
:10174000C98F0184B188C183F18841840021C1849B
:1017500042241472B848817808A8C17401E04DE1B0
:101760001BE002260675C821CC140C02D4E87A804E
:101770000705D5297B0E14300A7EF908A9087503E0
:10178000A90F0C1412002801D11698067060783C3D
:101790002870D030E1628A143D0A82A2884A82A26F
:1017A000790A75E2794A75207A8875E07EC875A055
:1017B0008B0883E08B4883208C8883608CC88321CE
:1017C00046243108A800F0A4F9787A08A94871B82D
:1017D0007A8871A08DC8140585206B0BC210050C8A
:1017E00090012018103F75387D0875B87D8875A860
:1017F00078C006C017401CC8758E486946028A0A20
:1018000087428A4A87827D08A90A77C27D4A770281
:101810007E8A77428B10A90A80828B4A80807F085B
:101820007104A900A4380432F9000A14487C494024
:101830001803907C30129900F05DF90398F97D80CF
:1018400030817003990922A0310A700121C170030F
:101850009800218166E18B490041660521C166013E
:101860006715996030C97E002904D07249816101F1
:101870002102E02ABA480981618175009981822498
:10188000400DF6F8022802D2012100F003F91220DF
:101890001B05F906280CD20A215F4A41438918FF2B
:1018A000318131497F890703D5FA7D7C23FCF89685
:1018B0001005FFF81699E035C41A01AE1818092072
:1018C00000F0FBF821460F31059100284ED020236F
:1018D0003E22002156241C06F6F806460A960317F7
:1018E00014986C1ED03A04200EE03C207070012049
:1018F0003071009870801620052CD0B01D5A240736
:10190000F2F8F87D7071AC201306D52146304609F7
:10191000310C3000F0E7F803E030460A12DD2025F4
:10192000C8100630461230053032DA1A12121A1474
:1019300006D0F8E08B309A16709A2813B083B87AE4
:10194000B077304600F0BFF83AE0287B7071DC20B9
:1019500007B01D00F0C2F8163006B4F83DE0149E42
:101960001A2EC23008A7F801210646019E120D9ECC
:10197000300470703198200BF87D820709D57171A1
:10198000B01D6A3004A5F80AB6400B30461DE0C011
:1019900007C00F7071B2129978100BB081208CF0D3
:1019A00081608C308278227462300483F806601281
:1019B0001660302477F81421017000994180B97DB8
:1019C000017100F075F81598807E022826D16078A4
:1019D0001499084322D0082C120B2C100461F81221
:1019E0002C1C0C61784170297881700FE0406404F0
:1019F0001C06C00600200A6E0512390412400C1D98
:101A000088031C0820B1A201000411A00510079949
:101A10008180397E81563C064AF80020171805104F
:101A20000640BA7047C004600D03B401480190013C
:101A3000BD919B02000C83E1980C837D9F0C700488
:101A400049FA010C8309D30C836D5B24933D9948BB
:101A50008290488355073083D59C3083397B18109A
:101A600027796D0100002101804180818070470A43
:101A70007802704B7843708A788270CA78C2700B93
:101A80007903714A7942711A20046802600E0F349A
:101A9000704740063414497B41700570F1F7F3FC40
:101AA0002068F1F7A4FB256003141B2400761C09B1
:101AB00080024080C10240062B066419F8B54E78BA
:101AC0004821F0B248432349214D41180C46AA7ED3
:101AD000A0340027282C22EDC3020010B5074CE0EB
:101AE00069000408D5FFF7F3FF05480078002802D5
:101AF000D10120C0032062100006115012C6580008
:0C1B0000049FF401000112AA01218400DE
:00000001FF
